:100000000C94CE020C9400000C9400000C940000A0
:100010000C9400000C9400000C9400000C94000060
:100020000C9400000C9400000C9400000C94000050
:100030000C9400000C9400000C9400000C94000040
:100040000C94AB1C0C9400000C9400000C94000069
:100050000C9400000C9400000C9400000C94000020
:100060000C9400000C9400000C9400000C94000010
:100070000C9400000C9400000C94571D0C9400008C
:100080000C94611D0C9400000C940000010000030E
:1000900051030102040810204080FEFDFBF7EFDF52
:1000A000BF7F252E306600252E316600252E326654
:1000B00000252E336600252E346600252E35660079
:1000C000252E3666000025306C640025316C6400F6
:1000D00025326C640025336C640025346C64002583
:1000E000356C640025366C640025376C6400253857
:1000F0006C640025396C640025306C750025316C0A
:10010000750025326C750025336C750025346C75CF
:100110000025356C750025366C750025376C75002B
:1001200025386C750025396C75004E075D07600732
:10013000A907BB07C207D307DA07E907F8070708CB
:100140000A080D0856085B08600865086A086F0809
:10015000740889088A08D10815095C099A09B40944
:10016000C509F909350A490A5D0A750A8D0AA50A01
:10017000BA0AC50AD00ADB0AE60AF10AFE0A080B27
:10018000120B220B320B420B520B5B0B640B6F0BEF
:100190007A0B850B900BB30BD60BF90B1C0C3F0C99
:1001A000620C7B0CB70CE70C2B0D500D8F0DC50DA1
:1001B000010E1D0E370E680E980EC70EE60E130FB9
:1001C000440F5B0FAF0FD40FF90F14103D105410F4
:1001D0006B1082109910B010C710DE10F5100C11C2
:1001E0003D119D11C211E311111229128B12C71278
:1001F000031320137713B2132F146214D414EF14C3
:100200007016E8166E1771177D178C17E6175718BA
:10021000C218301961198C19D719321A581A881A4C
:100220006E176E176E176E176E176E176E176E17A6
:100230006E176E176E176E176E176E176E176E1796
:100240006E176E176E176E176E176E176E176E1786
:100250006E176E176E176E176E176E176E176E1776
:100260006E176E176E176E176E176E176E176E1766
:100270006E176E176E176E176E176E176E176E1756
:100280006E176E176E176E176E176E176E176E1746
:100290006E176E176E176E176E176E176E176E1736
:1002A0006E176E176E176E176E176E176E176E1726
:1002B0006E176E176E176E176E176E176E176E1716
:1002C0006E176E176E176E176E176E176E176E1706
:1002D0006E176E176E176E176E176E176E176E17F6
:1002E0006E176E176E176E176E176E176E176E17E6
:1002F0006E176E176E176E176E176E176E176E17D6
:100300006E176E176E176E176E176E176E176E17C5
:100310006E176E176E176E176E176E176E176E17B5
:100320006E176E176E176E176E176E176E176E17A5
:100330006E176E176E176E176E176E176E176E1795
:100340006E176E176E176E176E176E176E176E1785
:100350006E17E31A461BF01B00000000C0C1C181EC
:100360000140C30103C00280C241C60106C007802C
:10037000C7410500C5C1C4810440CC010CC00D803B
:10038000CD410F00CFC1CE810E400A00CAC1CB8142
:100390000B40C90109C00880C841D80118C01980A4
:1003A000D9411B00DBC1DA811A401E00DEC1DF81AA
:1003B0001F40DD011DC01C80DC411400D4C1D5816B
:1003C0001540D70117C01680D641D20112C0138044
:1003D000D3411100D1C1D0811040F00130C0318033
:1003E000F1413300F3C1F28132403600F6C1F781AA
:1003F0003740F50135C03480F4413C00FCC1FD813B
:100400003D40FF013FC03E80FE41FA013AC03B80C3
:10041000FB413900F9C1F88138402800E8C1E98181
:100420002940EB012BC02A80EA41EE012EC02F802B
:10043000EF412D00EDC1EC812C40E40124C025806A
:10044000E5412700E7C1E68126402200E2C1E381C1
:100450002340E10121C02080E041A00160C0618013
:10046000A1416300A3C1A28162406600A6C1A78129
:100470006740A50165C06480A4416C00ACC1AD813A
:100480006D40AF016FC06E80AE41AA016AC06B8043
:10049000AB416900A9C1A88168407800B8C1B981A1
:1004A0007940BB017BC07A80BA41BE017EC07F80AB
:1004B000BF417D00BDC1BC817C40B40174C075806A
:1004C000B5417700B7C1B68176407200B2C1B38141
:1004D0007340B10171C07080B041500090C19181F2
:1004E0005140930153C052809241960156C05780AB
:1004F0009741550095C1948154409C015CC05D803A
:100500009D415F009FC19E815E405A009AC19B81C0
:100510005B40990159C058809841880148C0498082
:1005200089414B008BC18A814A404E008EC18F8128
:100530004F408D014DC04C808C41440084C1858169
:100540004540870147C046808641820142C04380C2
:100550008341410081C18081404048E1FA3ECDCCD9
:100560004C3D0AD7A33B6F12033A17B75138ACC5BD
:10057000A73601000000010003008C000400020205
:100580008E001400530A2A011400670A3E01060275
:100590007B0A52010400A80D72050000F894EE27B2
:1005A000ECBBF1E0F5BFE5BFE0936C00F8E1F1BD15
:1005B000E1BD8DE0A2E0BB27ED938A95E9F780E0ED
:1005C00090E1A0E0B1E0ED930197E9F7E6E7F5E00F
:1005D00085919591009761F0A591B5910590159041
:1005E000BF01F00105900D920197E1F7FB01F0CFFB
:1005F000EFEFEDBFE0E1EEBFC0E0D2E00C94F60615
:10060000E8810E945D320E941224E2E0E0939B00A8
:10061000E8EDE0939A00E6E0E0939D00E0E0E093EF
:100620009800929A0E94633221F4EFECE0939900D3
:1006300037C0E130A0E0FA0721F4E7E6E093990043
:100640002FC0E230A0E0FA0721F4E3E3E093990041
:1006500027C0E330A0E0FA0721F4E2E2E09399003A
:100660001FC0E430A0E0FA0721F4EFE0E093990026
:1006700017C0E530A0E0FA0721F4E7E0E093990025
:100680000FC0E630A0E0FA0721F4E3E0E093990020
:1006900007C0E730A0E0FA0719F4E1E0E093990021
:1006A00049C0E881EA93E8EAFDE0FA93EA930E9400
:1006B0001224E2E0EBB9E8EDEAB9E6E0E093950058
:1006C000E0E0E0939000189A0E94633219F4EFEC96
:1006D000E9B930C0E130A0E0FA0719F4E7E6E9B97A
:1006E00029C0E230A0E0FA0719F4E3E3E9B922C037
:1006F000E330A0E0FA0719F4E2E2E9B91BC0E43004
:10070000A0E0FA0719F4EFE0E9B914C0E530A0E081
:10071000FA0719F4E7E0E9B90DC0E630A0E0FA07FE
:1007200019F4E3E0E9B906C0E730A0E0FA0711F4F4
:10073000E1E0E9B921960895E0E0EBBBEFEFEABB19
:10074000E0E0E5BBEFEFE4BBE0EFE2BBE3E0E1BB01
:10075000EFE0E0936200E8E0E0936100E1E0E09325
:100760006500E0E1E0936400E0E0E0BFE4E0E3BFC7
:10077000E6E0E2BFE0E0E1BFE1E0E7BFE0E0E09318
:100780007D00E0E8E8B9E0E0E0BDECE9E0939A0D37
:10079000E0918E0DEE7FE160E0938E0DE5E6E09353
:1007A000980DE4E0E093990DE0E0E093A30DE2E022
:1007B000EA930E9400034424E1E05E2EE2E0E0932D
:1007C0000102E0B3E095AE2FEA2FE295EF70E093DF
:1007D0000002EFE1E1BDEFE0E1BD789408950E94F1
:1007E000963EE0E0E093510AE093520AE8E0F0E838
:1007F0000E9467320E94713C2E2F3F2F0E94703260
:1008000000E010E00217130710F00C94DF04A6E2DA
:10081000BAE0BF93AF930E94623CDF010E9478323E
:100820003196EA0FFB1FAF91BF91ED93FC93E091DE
:10083000260AF091270A0E94753CE150F040604082
:1008400070404E2F5F2F0E947F320E947832E2303C
:10085000A0E0FA0751F50E948732E091260AF09154
:10086000270AE491E17079F00E948F32FF93EF93B1
:10087000E081EF93A2E9B0E00E949632AF91EA2BBB
:10088000AF91BF910EC00E948F32FF93EF93E08132
:10089000EF93AAE9B0E00E949632AF91EA23AF91BC
:1008A000BF91EC930E947F3275C0E330A0E0FA075D
:1008B00021F0E430A0E0FA0779F40E948732A42FF7
:1008C000B52FAA5FBD4FE091260AF091270AE49167
:1008D000EC930E947F325EC0E530A0E0FA0721F081
:1008E000E630A0E0FA0789F40E948732E42FF52F62
:1008F0000E949E32E091260AF091270A0E94713CE4
:10090000ED93FC930E947F3245C0E730A0E0FA07E8
:1009100021F0E830A0E0FA0709F404C0E930A0E0D3
:10092000FA0789F40E948732E42FF52F0E94A5323E
:10093000E091260AF091270A0E94753C0E946C3CC7
:100940000E947F3227C0EA30A0E0FA0719F50E9422
:100950008732E091260AF091270AE491E03081F095
:10096000E42FF52F4F5F5F4FEA5FFD4FFF93EF934B
:100970000E9487323197E491AF91BF91EC93E9CF18
:10098000A6E0B2E0A40FB51FE0E0EC930E9487322E
:100990003197E491E091260AF091270AE491E13041
:1009A00049F4E091510AF091520A3196E093510ACC
:1009B000F093520A0E9487320F5F1F4F23CF0E948D
:1009C0009D3E269608951A930A93E52DF0E0E130B6
:1009D000A0E0FA0781F5909800E0013040F50E9410
:1009E000AC32A5E9BDE00E94B3320E94AC32ABE963
:1009F000BDE00E94BA32A3E9BDE00E94BA32A5EA86
:100A0000BDE00E94BA32A4EABDE00E94BA32A3EA75
:100A1000BDE00E94BF32E02F0E94C432FF93EF93EB
:100A2000E2E0EA93EF91FF9109950F5FD6CFE0E006
:100A3000E0930702A7C0E230A0E0FA0711F00C949F
:100A4000C205E0E0F0E8E093260AF093270A0E944E
:100A5000CE323297FA93EA93E2E0F0E8FA93EA931F
:100A60000E948F24DF01E091260AF091270A0E945C
:100A7000713CEA17FB0711F00C94BF050E94EF03CD
:100A8000EAE0F0E80E94673234900E94873200E08A
:100A9000031510F00C94B605E091260AF091270A90
:100AA000E491EF701E2FE12F0E94C432FF93EF9369
:100AB000E091260AF091270A3196E491EA93EF91AA
:100AC000FF9109950E94D632A3EABDE0AE0FBF1F89
:100AD000E091260AF091270AE491E295EF70EC93F9
:100AE0000E94D632ADE9BDE0AE0FBF1F0E94CE32EC
:100AF000ED93FC930E94D632ACE9BDE0AE0FBF1F70
:100B0000E091260AF091270A34960E94DD32AFE97F
:100B1000BDE0AE0FBF1FE091260AF091270A35967F
:100B20000E94DD32A6EABDE0AE0FBF1FE091260AAB
:100B3000F091270A3696ED93FC93E091260AF09106
:100B4000270A3696FF93EF930E94D632AFE9BDE0B5
:100B50000E94E0320E94703BAF91BF91EA0FFB1FF1
:100B6000E093260AF093270A0F5F92CFE0E0F0E8C7
:100B7000E093260AF093270A909A919803C0E1E047
:100B80005E2E919A452C8FC20E94983E00E010E0A4
:100B9000E32DF0E00E171F0710F00C94F2060E94F0
:100BA000E532A4EABDE00E94E032309711F00C94E7
:100BB000B9060E94E532ABE9BDE0AE0FBF1FEC9174
:100BC000EF930E94E532AFE9BDE0AE0FBF1FEC919D
:100BD000AF91AE1710F00C94B0060E94E532ABE96D
:100BE000BDE00E94E0320E94703B2E2F3F2F0E94FA
:100BF000E532A6EABDE00E94EC3231960E94F43262
:100C0000309711F00C9454060E94E532A3EABDE03F
:100C10000E94E0323097F9F40E94E532A6EABDE086
:100C20000E94F9320E940233A6EABDE00E94EC3233
:100C30000E9405330E940233A6EABDE00E94EC3216
:100C40000E941133A6EABDE00E94EC320E941D33DF
:100C50000E94233322C0E130A0E0FA07F1F40E94A1
:100C6000E532A6EABDE00E94F9320E94E532A6EA2A
:100C7000BDE00E94EC320E9405330E94E532A6EAF4
:100C8000BDE00E94EC320E941133A6EABDE00E9452
:100C9000EC320E941D330E9429330E94E532A5EAFE
:100CA000BDE00E942F3355C0E130A0E0FA0711F0FB
:100CB0000C94A9060E94E532A3EABDE00E94E0324E
:100CC0003097F9F40E94E532A6EABDE00E94F932BD
:100CD0000E940233A6EABDE00E94EC320E94053376
:100CE0000E940233A6EABDE00E94EC320E9411335A
:100CF000A6EABDE00E94EC320E941D330E9434330C
:100D000022C0E130A0E0FA07F1F40E94E532A6EA41
:100D1000BDE00E94F9320E94E532A6EABDE00E94E1
:100D2000EC320E9405330E94E532A6EABDE00E9443
:100D3000EC320E941133A6EABDE00E94EC320E9420
:100D40001D330E943A330E94E532A5EABDE00E94BD
:100D500040330E94E532ABE9BDE00E94453307C055
:100D60000E94E532ABE9BDE0AE0FBF1FE0E0EC93BF
:100D700036C0E530A0E0FA0729F40E94E5320E946F
:100D80004A332DC0E630A0E0FA0749F50E94E5326B
:100D9000A3E9BDE00E944533EC93EF930E94E53256
:100DA000ACE9BDE0AE0FBF1FEC91AF91AE1748F4B8
:100DB0000E94E532ABE9BDE0AE0FBF1FEC91E15000
:100DC00007C00E94E532A3E9BDE0AE0FBF1FE0E01F
:100DD000EC930E94E532A4EABDE00E94BF320F5FAF
:100DE0001F4FD6CE0E949F3E249608950E949C03DA
:100DF0000E94271C0E94341CE52DA42D0E948E3BCE
:100E0000EF93A091A40DE0E00E94933BAF91EA2BF9
:100E100011F40C944A07E42DF0E0E130A0E0FA0769
:100E200011F500E0013080F40E94AC32A4EABDE08C
:100E3000AE0FBF1FAC91A53029F4E02F0E945033B4
:100E40000E944A330F5FEECFE0916300E17039F406
:100E5000A0910102A23011F4E2E05E2E03C0E2E0B4
:100E6000E093010216C0E230A0E0FA0791F40E947C
:100E7000131C0E94C405E0916300E170EF93A09100
:100E80000102E1E00E948E3BAF91EA2B11F0E1E01C
:100E90005E2E02C00E94E304ADCFFFCFE1E0F0E0A0
:100EA00060E070E0E093490AF0934A0A60934B0ACD
:100EB00070934C0A0E947F3208950E947F320895F9
:100EC0000E9456330E94593317FF21C010700E94B0
:100ED0005F33E081EF930E946833AF91EA2369F0BA
:100EE000E1E0F0E060E070E0E093490AF0934A0A44
:100EF00060934B0A70934C0A09C0E0E0E093490A02
:100F0000E0934A0AE0934B0AE0934C0A21C0015057
:100F100010400E947233E081EF930E946833AF91DA
:100F2000EA2369F0E1E0F0E060E070E0E093490A74
:100F3000F0934A0A60934B0A70934C0A09C0E0E0B0
:100F4000E093490AE0934A0AE0934B0AE0934C0A83
:100F5000AAC00E947F320E947933F0E0E7FDFFEFE4
:100F60000E94843BE093490AF0934A0A60934B0A3B
:100F700070934C0A08950E947F320E9479330E9438
:100F8000813308950E947F320E948D330E94623C1B
:100F90000E94843BE093490AF0934A0A60934B0A0B
:100FA00070934C0A08950E947F320E948D330E94F4
:100FB000923308950E947F320E949F330E94663CC4
:100FC000E093490AF0934A0A60934B0A70934C0AE3
:100FD00008950E947F320E949F330E94663CE093F6
:100FE000490AF0934A0A60934B0A70934C0A089599
:100FF0000E947F320E949F330E94663CE0934D0A1C
:10100000F0934E0A60934F0A7093500A08950E941D
:101010007F3208950E947F3208950E9456330E94C5
:10102000593317FF20C01070E091490AE17069F050
:101030000E945F33FF93EF93E081EF930E94683348
:10104000AF91EA2BAF91BF910CC00E945F33FF9329
:10105000EF93E081EF930E94A433AF91EA23AF9125
:10106000BF91EC9320C001501040E091490AE1701B
:1010700069F00E947233FF93EF93E081EF930E9437
:101080006833AF91EA2BAF91BF910CC00E947233CD
:10109000FF93EF93E081EF930E94A433AF91EA2393
:1010A000AF91BF91EC930991199108950E947F32FD
:1010B0000E94AE3308950E947F320E94AE3308959D
:1010C0000E947F320E94BF3308950E947F320E94A7
:1010D000BF3308950E947F320E94D43308950E9446
:1010E0007F320E94D43308950E947F320E94E933F8
:1010F000A6E0B2E00E94723BAE0FBF1FE0914D0A26
:10110000F0914E0A60914F0A7091500A0E946C3C17
:101110000895089524970E9456330E9487320E94B2
:10112000EE3341F1EFEFFFEF6FEF7FEFEA83FB83E9
:101130006C837D8300E0011760F40E940D340E94EF
:1011400015340E94403BEA83FB836C837D830F5FF1
:10115000F2CF0E942B340E943834E1E0F0E060E0EE
:1011600070E0E093490AF0934A0A60934B0A709347
:101170004C0A12C0A6E2BAE0BF93AF930E94423479
:10118000AF91BF910E944C3429F00E940D340E940F
:10119000383402C00E947F320E940D340E943834DD
:1011A00087C024970E9456330E9487320E94EE33F4
:1011B00029F1E0E0EA83EB83EC83ED8300E00117A3
:1011C00060F40E940D340E9415340E94453BEA836E
:1011D000FB836C837D830F5FF2CF0E942B340E94D0
:1011E0003834E1E0F0E060E070E0E093490AF09329
:1011F0004A0A60934B0A70934C0A12C0A6E2BAE006
:10120000BF93AF930E944234AF91BF910E944C3480
:1012100029F00E940D340E94383402C00E947F32AF
:101220000E940D340E94383443C024970E945633E4
:101230000E9487320E94EE3329F1E0E0EA83EB83DB
:10124000EC83ED8300E0011760F40E940D340E94EE
:1012500015340E944A3BEA83FB836C837D830F5FD6
:10126000F2CF0E942B340E943834E1E0F0E060E0DD
:1012700070E0E093490AF0934A0A60934B0A709336
:101280004C0A12C0A6E2BAE0BF93AF930E94423468
:10129000AF91BF910E944C3429F00E940D340E94FE
:1012A000383402C00E947F320E940D340E943834CC
:1012B00019810881269608950E947F320E940D347C
:1012C0000E9456340E947E3EF9F00E940D340E9426
:1012D00056340E94893BE093490AF0934A0A60938E
:1012E0004B0A70934C0A0E940D340E943834E1E09E
:1012F000F0E060E070E0E093490AF0934A0A6093FE
:101300004B0A70934C0A11C00E947F32E091260A6A
:10131000F091270A0E94713CF07829F00E940D3468
:101320000E94383402C00E947F320E940D340E9415
:10133000383408950E947F320E940D340E94563442
:101340000E947E3E71F0E0E0E093490AE0934A0A91
:10135000E0934B0AE0934C0A0E940D340E9438340B
:1013600002C00E947F3208950E947F320E940D3495
:101370000E9456340E947E3E29F00E940D340E9445
:10138000383402C00E947F3208950E947F320E944A
:101390000D340E9456340E947E3E11F10E940D349D
:1013A0000E9456340E947E3E89F4E1E0F0E060E065
:1013B00070E0E093490AF0934A0A60934B0A7093F5
:1013C0004C0A0E9468340E94383409C0E0E0E0937F
:1013D000490AE0934A0AE0934B0AE0934C0A04C09E
:1013E0000E940D340E9438340E940D340E9438341B
:1013F00008950E947F320E940D340E9456340E944C
:101400007E3E09F50E940D340E9456340E947E3EB5
:10141000C9F0E0E0E093490AE0934A0AE0934B0AFE
:10142000E0934C0A0E9468340E943834E1E0F0E016
:1014300060E070E0E093490AF0934A0A60934B0A37
:1014400070934C0A0DC00E940D340E943834E0E0C5
:10145000E093490AE0934A0AE0934B0AE0934C0A6E
:101460000E940D340E943834089524970E947F32E0
:101470000E940D340E945634E883F9836A837B838B
:101480000E940D340E9456340E9470340E943834F9
:101490006FC024970E947F320E940D340E94563400
:1014A000E883F9836A837B830E940D340E9456345B
:1014B0000E9482340E9438345BC024970E947F329D
:1014C0000E940D340E945634E883F9836A837B833B
:1014D0000E940D340E945634A881B9818A819B8173
:1014E0000E9494340E94383443C024970E947F3273
:1014F0000E940D340E945634E883F9836A837B830B
:101500000E940D340E945634A881B9818A819B8142
:101510000E94A2340E9438342BC024970E947F324C
:101520000E940D340E945634E883F9836A837B83DA
:101530000E940D340E945634A881B9818A819B8112
:101540000E94B0340E94383413C024970E947F3226
:101550000E940D340E945634E883F9836A837B83AA
:101560000E940D340E9456340E94BE340E943834CA
:10157000249608950E947F320E940D340E94D03438
:101580000E94E6340E94383408950E947F320E94FF
:101590000D340E94D0340E94F4340E9438340895EF
:1015A0000E947F320E940D340E94D0340E949434F5
:1015B0000E94383408950E947F320E940D340E94A8
:1015C000D0340E94A2340E94383408950E947F32A1
:1015D0000E940D340E94D0340E94B0340E943834EE
:1015E00008950E947F320E940D340E94D0340E94E0
:1015F000B03B0E9402350E943834089524970E941F
:101600007F320E940E350E9470340E94383446C2E8
:1016100024970E947F320E940E350E9482340E94DD
:1016200038343CC224970E947F320E940E35A88134
:10163000B9818A819B810E94723E0E9402350E947C
:1016400038342CC224970E947F320E940E35A88124
:10165000B9818A819B810E94783E0E9402350E9456
:1016600038341CC224970E947F320E940E35A88114
:10167000B9818A819B810E94663E0E9402350E9448
:1016800038340CC224970E947F320E940E35A88104
:10169000B9818A819B810E946C3E0E9402350E9422
:1016A0003834FCC10E947F320E9427350E94E63404
:1016B0000E94383408950E947F320E9427350E948C
:1016C000F4340E94383408950E947F320E942735F6
:1016D0000E94723E0E9402350E94383408950E9492
:1016E0007F320E9427350E94783E0E9402350E9478
:1016F000383408950E947F320E9427350E94663E4A
:101700000E9402350E94383408950E947F320E9460
:1017100027350E946C3E0E9402350E94383408959D
:101720000E947F320E940D340E9456340E947E3EF9
:1017300099F00E940D340E9436350E945608E1E06F
:10174000F0E060E070E0E093490AF0934A0A6093A9
:101750004B0A70934C0A02C00E9440350E940D341F
:101760000E94383408950E947F320E940D340E94F6
:1017700056340E947E3E99F00E940D340E94363508
:101780000E946008E1E0F0E060E070E0E093490A68
:10179000F0934A0A60934B0A70934C0A02C00E946D
:1017A00040350E940D340E94383408950E947F32E3
:1017B0000E940D340E9456340E947E3E99F00E9491
:1017C0000D340E9436350E946A08E1E0F0E060E0E6
:1017D00070E0E093490AF0934A0A60934B0A7093D1
:1017E0004C0A02C00E9440350E940D340E943834D9
:1017F00008950E947F320E940D340E9456340E9448
:101800007E3E99F00E940D340E9436350E945B089E
:10181000E1E0F0E060E070E0E093490AF0934A0A0A
:1018200060934B0A70934C0A02C00E9440350E949C
:101830000D340E94383408950E947F320E940D3486
:101840000E9456340E947E3E99F00E940D340E9400
:1018500036350E946508E1E0F0E060E070E0E0937A
:10186000490AF0934A0A60934B0A70934C0A02C0EB
:101870000E9440350E940D340E94383408950E9421
:101880007F320E940D340E9456340E947E3E99F0B1
:101890000E940D340E9436350E946F08E1E0F0E0AE
:1018A00060E070E0E093490AF0934A0A60934B0AC3
:1018B00070934C0A02C00E9440350E940D340E9471
:1018C000383408950E947F320E940D340E945634AD
:1018D0000E947E3E49F00E940D340E9456340E94C0
:1018E000473D0E94483502C00E9440350E940D3499
:1018F0000E943834089524970E9456330E948732FC
:101900000E94EE3329F1E0E0EA83EB83EC83ED8380
:1019100000E0011760F40E940D340E9415340E940B
:10192000363BEA83FB836C837D830F5FF2CF0E949B
:101930002B340E943834E1E0F0E060E070E0E093A6
:10194000490AF0934A0A60934B0A70934C0A0AC002
:10195000A6E2BAE0BF93AF930E945F35AF91BF910B
:10196000ED93FC930E940D340E9438340AC12497F1
:101970000E9456330E9487320E94EE33C9F0E0E0A5
:10198000EA83EB83EC83ED8300E0011750F40E94BF
:101990006A350E94853DEA83FB836C837D830F5FFC
:1019A000F4CFEA81FB816C817D810E9448350AC0B9
:1019B000A6E2BAE0BF93AF930E945F35AF91BF91AB
:1019C000ED93FC930E940D340E943834DAC02497C2
:1019D0000E947F320E940D340E9456340E947E3E47
:1019E00099F10E940D340E945634E883F9836A838A
:1019F0007B830E940D340E943635A091490AB09134
:101A00004A0A80914B0A90914C0AE881F9816A81D7
:101A10007B810E943B3BE093490AF0934A0A609322
:101A20004B0A70934C0A0E940D340E943834E1E056
:101A3000F0E060E070E0E093490AF0934A0A6093B6
:101A40004B0A70934C0A02C00E9479350E940D34F3
:101A50000E94383423C024970E947F320E940D34A4
:101A60000E9456340E947E3E99F00E948135A091DA
:101A70004D0AB0914E0A80914F0A9091500AE88128
:101A8000F9816A817B810E947E3D0E94483502C0B7
:101A90000E9479350E940D340E94383424960895AE
:101AA00024970E9456330E9487320E94EE3341F100
:101AB000E1E0F0E060E070E0EA83FB836C837D832B
:101AC00000E0011760F40E940D340E9415340E945A
:101AD000F03BEA83FB836C837D830F5FF2CF0E9430
:101AE0002B340E943834E1E0F0E060E070E0E093F5
:101AF000490AF0934A0A60934B0A70934C0A0AC051
:101B0000A6E2BAE0BF93AF930E945F35AF91BF9159
:101B1000ED93FC930E940D340E94383432C0249718
:101B20000E9456330E9487320E94EE33E1F0E0E0DB
:101B3000F0E060E87FE3EA83FB836C837D8300E071
:101B4000011750F40E946A350E94D33DEA83FB835B
:101B50006C837D830F5FF4CFEA81FB816C817D8193
:101B60000E9448350AC0A6E2BAE0BF93AF930E9434
:101B70005F35AF91BF91ED93FC930E940D340E94AD
:101B80003834198108812696089524970E947F325F
:101B90000E940D340E9456340E947E3E59F10E94EC
:101BA0000D340E945634E883F9836A837B830E9454
:101BB0000D340E945634A881B9818A819B810E948C
:101BC0002E3CE093490AF0934A0A60934B0A7093C3
:101BD0004C0A0E940D340E943834E1E0F0E060E0ED
:101BE00070E0E093490AF0934A0A60934B0A7093BD
:101BF0004C0A02C00E9479350E940D340E9438348C
:101C000011C224970E947F320E940D340E945634E4
:101C10000E947E3E59F00E940E35A881B9818A81CA
:101C20009B810E94053E0E94483502C00E94793582
:101C30000E940D340E943834F5C124970E947F32EF
:101C40000E940D340E9456340E947E3E49F00E944C
:101C500081350E9491350E94372D0E94483502C07F
:101C60000E9479350E940D340E943834DBC10E94F5
:101C70007F320E940D340E9456340E947E3E09F14C
:101C80000E940D340E945634EF5FFF4F6F4F7F4F1D
:101C9000E093490AF0934A0A60934B0A70934C0A06
:101CA0000E940D340E943834E1E0F0E060E070E022
:101CB000E093490AF0934A0A60934B0A70934C0AE6
:101CC00002C00E9440350E940D340E9438340895AD
:101CD0000E947F320E940D340E9456340E947E3E44
:101CE00001F10E940D340E945634319760407040DB
:101CF000E093490AF0934A0A60934B0A70934C0AA6
:101D00000E940D340E943834E1E0F0E060E070E0C1
:101D1000E093490AF0934A0A60934B0A70934C0A85
:101D200002C00E9440350E940D340E94383408954C
:101D30000E947F320E940D340E9456340E947E3EE3
:101D4000F9F00E940D340E9456340E944F3BE093FC
:101D5000490AF0934A0A60934B0A70934C0A0E9416
:101D60000D340E943834E1E0F0E060E070E0E09390
:101D7000490AF0934A0A60934B0A70934C0A02C0D6
:101D80000E9440350E940D340E94383408950E940C
:101D90007F320E940D340E9456340E947E3E79F0BC
:101DA0000E94F807E0914D0AF0914E0A60914F0AA7
:101DB0007091500A0E94EB3C0E94483502C00E947C
:101DC00040350E940D340E94383408950E947F32BD
:101DD0000E940D340E9456340E947E3EE9F00E941B
:101DE0003F320E94843BE093490AF0934A0A609391
:101DF0004B0A70934C0A0E940D340E943834E1E083
:101E0000F0E060E070E0E093490AF0934A0A6093E2
:101E10004B0A70934C0A02C00E947F320E940D341C
:101E20000E94383408950E947F320E940D340E942F
:101E300056340E947E3E09F10E940D340E945634B1
:101E40000E947B3C0E940C2DE093490AF0934A0AC1
:101E500060934B0A70934C0A0E940D340E943834F0
:101E6000E1E0F0E060E070E0E093490AF0934A0AB4
:101E700060934B0A70934C0A02C00E9440350E9446
:101E80000D340E94383408950E947F320E940D3430
:101E90000E9456340E947E3E39F00E94A2350E9474
:101EA000312D0E94483502C00E9440350E940D34F9
:101EB0000E943834089524970E947F320E940D3486
:101EC0000E9456340E947E3E11F40C94A80F0E948A
:101ED000A2350E94233BE883F9836A837B83A09128
:101EE0004D0AB0914E0A80914F0A9091500A0E947B
:101EF000AF350E94463E28F4E881F9816A817B81F2
:101F00000CC0E0914D0AF0914E0A60914F0A709119
:101F1000500A0E947B3C0E94293B0E94143DE093A2
:101F2000490AF0934A0A60934B0A70934C0A0E9444
:101F30000D340E943834E1E0F0E060E070E0E093BE
:101F4000490AF0934A0A60934B0A70934C0A02C004
:101F50000E9440350E940D340E94383463C00E94B4
:101F60007F320E940D340E9456340E947E3EA9F0BA
:101F70000E94A2350E94293B0E94BA350E94383443
:101F8000E1E0F0E060E070E0E093490AF0934A0A93
:101F900060934B0A70934C0A02C00E9440350E9425
:101FA0000D340E94383408950E947F320E940D340F
:101FB0000E9456340E947E3EA9F00E94A2350E94E3
:101FC000233B0E94BA350E943834E1E0F0E060E043
:101FD00070E0E093490AF0934A0A60934B0A7093C9
:101FE0004C0A02C00E9440350E940D340E943834D1
:101FF000089524970E947F320E940D340E94563427
:102000000E947E3E49F00E9481350E9491350E94D7
:10201000CD2E0E94483502C00E9479350E940D34B1
:102020000E943834249608950E947F320E940D3415
:102030000E9456340E947E3EC9F00E940D340E94D8
:1020400056340E947B3C0E941D2D0E94C5350E9483
:102050003834E1E0F0E060E070E0E093490AF093AA
:102060004A0A60934B0A70934C0A02C00E944035A2
:102070000E940D340E94383408950E947F320E94DD
:102080000D340E9456340E947E3E39F00E94A235E3
:102090000E94BE3A0E94483502C00E9440350E940C
:1020A0000D340E94383408950E947F320E940D340E
:1020B0000E9456340E947E3E39F00E94A2350E9452
:1020C000212E0E94483502C00E9440350E940D34E6
:1020D0000E94383408950E947F320E940D340E947D
:1020E00056340E947E3E39F00E94A2350E94852D12
:1020F0000E94483502C00E9440350E940D340E9463
:10210000383408950E947F320E940D340E94563464
:102110000E947E3E39F00E94A2350E942D2F0E941F
:10212000483502C00E9440350E940D340E94383468
:1021300008950E947F320E940D340E9456340E94FE
:102140007E3E39F00E94A2350E94BE2F0E94483583
:1021500002C00E9440350E940D340E943834089518
:102160000E947F320E940D340E9456340E947E3EAF
:1021700039F00E94A2350E94CD2F0E94483502C03E
:102180000E9440350E940D340E94383408950E9408
:102190007F320E940D340E9456340E947E3E39F0F8
:1021A0000E94A2350E9486300E94483502C00E94DB
:1021B00040350E940D340E94383408950E947F32C9
:1021C0000E940D340E9456340E947E3E39F00E94D7
:1021D000A2350E94F5300E94483502C00E94403569
:1021E0000E940D340E94383408950E947F320E946C
:1021F0000D340E9456340E947E3E39F00E94A23572
:102200000E941B310E94483502C00E9440350E9446
:102210000D340E94383408950E947F320E940D349C
:102220000E9456340E947E3E09F1E091810CF091AB
:10223000820C6091830C7091840CE093490AF093B6
:102240004A0A60934B0A70934C0A0E940D340E9414
:102250003834E1E0F0E060E070E0E093490AF093A8
:102260004A0A60934B0A70934C0A02C00E947F3264
:102270000E940D340E943834089524970E947F32C2
:102280000E940D340E9456340E947E3E11F40C943C
:1022900088110E940D340E943635A091490AB091F0
:1022A0004A0A80914B0A90914C0AE091810CF0917E
:1022B000820C6091830C7091840C0E943B3BE883FC
:1022C000F9836A837B830E940D340E9456340E94F6
:1022D000BE340E943834E881F9816A817B81E093C1
:1022E000490AF0934A0A60934B0A70934C0A0E9481
:1022F0000D340E943834E1E0F0E060E070E0E093FB
:10230000490AF0934A0A60934B0A70934C0A10C032
:102310000E94D0350E944C3439F00E940D340E9446
:1023200038340E94D63502C00E94D035ED93FC931C
:102330000E940D340E94383481C10E947F320E9475
:102340000D340E9456340E947E3EA9F00E940D3446
:102350000E9436350E940D340E943834E1E0F0E0EE
:1023600060E070E0E093490AF0934A0A60934B0AF8
:1023700070934C0A02C00E9440350E940D340E94A6
:10238000383408950E947F320E940D340E945634E2
:102390000E947E3E89F00E94F8070E947408E1E0E6
:1023A000F0E060E070E0E093490AF0934A0A60933D
:1023B0004B0A70934C0A02C00E9440350E940D34B3
:1023C0000E94383408950E947F320E940D340E948A
:1023D00056340E947E3EF1F00E947F3234970E9474
:1023E000753CE093490AF0934A0A60934B0A709354
:1023F0004C0A0E940D340E943834E1E0F0E060E0C5
:1024000070E0E093490AF0934A0A60934B0A709394
:102410004C0A02C00E9440350E940D340E9438349C
:1024200008950E947F320E940D340E9456340E940B
:102430007E3E41F00E947F3234970E94753C0E949C
:10244000483502C00E9440350E940D340E94383445
:10245000089522970E94963E26E032E00E947F3245
:102460000E940D340E9456340E947E3E11F40C945A
:1024700081120E940D340E9436350091490A109154
:102480004A0A0E940D340E943635E091490AF091C3
:102490004A0AEE83FF83E091260AF091270A0E9400
:1024A000713C0E0F1F1F0E947F320E940D340E944C
:1024B0003635E091490AF0914A0A2E0F3F1F40E05D
:1024C00050E0EE81FF814E175F0770F4E42FF52F87
:1024D0000E94DC353196E050F048E00FF11FE491A6
:1024E000EC934F5F5F4FEDCFE1E0F0E060E070E034
:1024F000E093490AF0934A0A60934B0A70934C0A9E
:1025000002C00E94E2350E940D340E9438340E94BD
:102510009D3E2896089524970E947F320E940D3494
:102520000E9456340E947E3E59F10E940D340E9452
:102530005634E883F9836A837B830E940D340E94BA
:102540005634A881B9818A819B810E94643BE093C3
:10255000490AF0934A0A60934B0A70934C0A0E940E
:102560000D340E943834E1E0F0E060E070E0E09388
:10257000490AF0934A0A60934B0A70934C0A02C0CE
:102580000E9479350E940D340E94383457C0249738
:102590000E947F320E940D340E9456340E947E3E7B
:1025A00059F10E940D340E945634E883F9836A83FE
:1025B0007B830E940D340E945634A881B9818A81A0
:1025C0009B810E94583BE093490AF0934A0A60932A
:1025D0004B0A70934C0A0E940D340E943834E1E09B
:1025E000F0E060E070E0E093490AF0934A0A6093FB
:1025F0004B0A70934C0A02C00E9479350E940D3438
:102600000E9438341BC024970E947F320E940D34F0
:102610000E9456340E947E3E59F00E947F320E94F2
:10262000E9330E94EA350E9439310E94483502C0E0
:102630000E9440350E940D340E943834249608953B
:102640000A930E947F320E940D340E9456340E94E9
:102650007E3E11F40C946F130E94F8070E940D3413
:102660000E9436350091490AE6E0E01708F406E0DA
:102670000E947F320E94E93366277727E093490A58
:10268000F0934A0A60934B0A70934C0A0E94F53506
:10269000E2EAF0E0FF93EF930E940236AF91BF9120
:1026A000EA0FFB1FFA93EA93E0914D0AF0914E0A6C
:1026B00060914F0A7091500A0E947B3C84E00E9416
:1026C000C02B2896E1E0F0E060E070E0E093490A7A
:1026D000F0934A0A60934B0A70934C0A02C00E941E
:1026E00079350E940D340E943834099108950E9472
:1026F0007F320E940D340E9456340E947E3E51F17A
:10270000A8E4BAE0EC91F0E0EF5FEC93E1500E94B6
:102710000936DF01E6E2FAE082E00E94C43C0E9452
:102720000F3620FE05C00E9470320E941C36F9CF81
:10273000689420F8E091480AE150E093480AEF5F7E
:10274000A8E4BAE0EC910E940936A6E2BAE082E081
:102750000E94C43CA6E2BAE00E94623C3496ED932B
:10276000FC93089526970E947F320E940D340E94A8
:1027700056340E947E3E11F40C9428140E940D34AD
:10278000E330A0E0FA0721F0E430A0E0FA07C9F452
:102790000E940D340E945634E883F9836A837B8358
:1027A0000E940D340E943635E091490AF0914A0AA0
:1027B000EC83FD83AC81BD811197E8810E94B53C1B
:1027C0003AC0E530A0E0FA0721F0E630A0E0FA07D1
:1027D000E1F40E940D340E945634E883F9836A8341
:1027E0007B830E940D340E943635E091490AF091B6
:1027F0004A0AEE0FFF1FEC83FD83AC81BD81129767
:10280000E881F9810E94AD3C16C0E730A0E0FA07EC
:1028100021F0E830A0E0FA0771F40E940D340E9424
:102820005634E883F9836A837B830E940D340E94C7
:1028300036350E942936E1E0F0E060E070E0E09398
:10284000490AF0934A0A60934B0A70934C0A02C0FB
:102850000E9440350E940D340E94383431C02697C2
:102860000E947F320E940D340E9456340E947E3EA8
:1028700009F10E94F807E0914D0AF0914E0A60912B
:102880004F0A7091500AE883F9836A837B830E9420
:102890000D340E9436350E942936E1E0F0E060E018
:1028A00070E0E093490AF0934A0A60934B0A7093F0
:1028B0004C0A02C00E9440350E940D340E943834F8
:1028C0002696089522970E947F320E940D340E941E
:1028D00056340E947E3E11F40C94CD140E940D34A7
:1028E0000E9436350E940D34E330A0E0FA0721F053
:1028F000E430A0E0FA0771F4E091490AF0914A0A45
:10290000E883F983A881B98111970E94963C0E94BF
:10291000813332C0E530A0E0FA0721F0E630A0E0D4
:10292000FA07C1F4E091490AF0914A0AEE0FFF1F3D
:10293000E883F983A881B98112970E94923C6627A7
:102940007727E093490AF0934A0A60934B0A709301
:102950004C0A12C0E730A0E0FA0721F0E830A0E00E
:10296000FA0751F40E943B36E093490AF0934A0A71
:1029700060934B0A70934C0A0E940D340E943834C5
:10298000E1E0F0E060E070E0E093490AF0934A0A89
:1029900060934B0A70934C0A02C00E9440350E941B
:1029A0000D340E94383419C022970E947F320E9451
:1029B0000D340E9456340E947E3E49F00E940D3430
:1029C0000E9436350E943B360E94483502C00E9464
:1029D00040350E940D340E94383422960895EC97B9
:1029E0000E947F320E940D340E9456340E947E3E27
:1029F00011F40C9463160E940D340E945634ECAB13
:102A0000FDAB6EAB7FAB0E940D340E945634E8AB39
:102A1000F9AB6AAB7BAB0E940D340E945634ECA735
:102A2000FDA76EA77FA70E940D340E945634E8A729
:102A3000F9A76AA77BA70E940D340E945634ECA325
:102A4000FDA36EA37FA30E940D340E945634E8A319
:102A5000F9A36AA37BA30E940D340E945634EC8F25
:102A6000FD8F6E8F7F8F0E940D340E945634E88F49
:102A7000F98F6A8F7B8F0E940D340E945634EC8B45
:102A8000FD8B6E8B7F8B0E940D340E945634EC8739
:102A9000FD876E877F87A091810CB091820C809119
:102AA000830C9091840C0E94803C0E943B3BE88BFD
:102AB000F98B6A8B7B8BE091810CF091820C609199
:102AC000830C7091840CEC87FD876E877F87A889C3
:102AD000B9898A899B890E94863E44F0E1E0F0E052
:102AE00060E070E0E88BF98B6A8B7B8BA8A9B9A9B1
:102AF0008AA99BA9ECA9FDA96EA97FA90E943B3BCD
:102B0000E8AFF9AF6AAF7BAFACA5BDA58EA59FA519
:102B10000E94F03BE887F9876A877B87E889F98913
:102B20006A897B89A8ADB9AD8AAD9BAD0E94F03BA7
:102B3000A8A5B9A58AA59BA50E94F03BA88DB98D33
:102B40008A8D9B8D0E94363BEC83FD836E837F8351
:102B5000EC8DFD8D6E8D7F8DAC81BD818E819F81D1
:102B60000E948C3E24F4EC83FD836E837F83E8A176
:102B7000F9A16AA17BA1AC81BD818E819F810E9458
:102B8000913E24F4EC83FD836E837F83AC89BD8901
:102B90008E899F89E8ADF9AD6AAD7BAD0E943B3B64
:102BA000ACA1BDA18EA19FA10E94F03BDF01CB0192
:102BB000E889F9896A897B890E942E3CE883F98338
:102BC0006A837B83EC81FD816E817F81A885B985D5
:102BD0008A859B850E944936E093490AF0934A0A08
:102BE00060934B0A70934C0AEC8DFD8D6E8D7F8D3A
:102BF000A091490AB0914A0A80914B0A90914C0ADF
:102C00000E948C3E44F4E093490AF0934A0A609390
:102C10004B0A70934C0AE8A1F9A16AA17BA1A0918B
:102C2000490AB0914A0A80914B0A90914C0A0E943D
:102C3000913E44F4E093490AF0934A0A60934B0AA8
:102C400070934C0A0E940D340E943834EC81FD814F
:102C50006E817F81E093490AF0934A0A60934B0AA0
:102C600070934C0A0E940D340E943834E8ADF9ADDF
:102C70006AAD7BADE093490AF0934A0A60934B0A30
:102C800070934C0A0E940D340E943834EC85FD8507
:102C90006E857F85E093490AF0934A0A60934B0A58
:102CA00070934C0A0E940D340E943834E1E0F0E049
:102CB00060E070E0E093490AF0934A0A60934B0A9F
:102CC00070934C0A07C0A6E2BAE00E94623CF896F4
:102CD000ED93FC930E940D340E943834EC960895D5
:102CE00024970A930E947F320E940D340E9456342A
:102CF0000E947E3E11F40C94DF160E947F320E94E7
:102D0000E93366277727E983FA836B837C830E9404
:102D10000D340E9436350091490AE9E0E01708F4C5
:102D200009E00E940D34E330A0E0FA0721F0E5301D
:102D3000A0E0FA0709F404C0E730A0E0FA0789F43C
:102D40000E945236E6ECF0E0FF93EF930E940236C9
:102D5000AF91BF910E945B3684E00E94012D2896BE
:102D60001DC0E430A0E0FA0721F0E630A0E0FA0749
:102D700009F404C0E830A0E0FA0781F40E9452365A
:102D8000E8EFF0E0FF93EF930E940236AF91BF911E
:102D90000E945B3684E00E94012D28960E940D342B
:102DA0000E943834E1E0F0E060E070E0E093490A2E
:102DB000F0934A0A60934B0A70934C0A02C00E9437
:102DC00079350E940D340E94383408812596089583
:102DD00024970E9456330E940D340E9456340E945C
:102DE0007E3E11F40C946417E091260AF091270AB4
:102DF00033960491E02FF0E00E945634EA83FB837F
:102E00006C837D830E940D340E9436351091490AEF
:102E1000E9E0E11708F419E00E947F320E94E933EB
:102E200066277727E093490AF0934A0A60934B0A92
:102E300070934C0AE02FF0E0E330A0E0FA0721F0B5
:102E4000E530A0E0FA0709F404C0E730A0E0FA0793
:102E500089F40E94F535E6ECF0E0FF93EF930E94D1
:102E60006636AF91BF910E946D3684E00E94C02B00
:102E700028961DC0E430A0E0FA0721F0E630A0E07B
:102E8000FA0709F404C0E830A0E0FA0781F40E94D0
:102E9000F535E8EFF0E0FF93EF930E946636AF91CF
:102EA000BF910E946D3684E00E94C02B2896E1E01D
:102EB000F0E060E070E0E093490AF0934A0A609322
:102EC0004B0A70934C0A02C00E9479350E940D345F
:102ED0000E9438341981088126960895E89420F8D4
:102EE00008950E947F320E940D340E9456340E9441
:102EF0007E3E11F0E89420F808950E947F320E94EF
:102F00000D340E9456340E947E3E19F00E940F3606
:102F100002C00E947F32089522970E94963E06E0EA
:102F200012E026E032E00E947F320E940D340E94BF
:102F300056340E947E3E11F40C94DD170E940D342D
:102F40000E943635E091490AF0914A0A0E0F1F1F80
:102F50000E940D340E943635E091490AF0914A0AE8
:102F6000EE83FF830E940D340E943635E091490ABA
:102F7000F0914A0A2E0F3F1F40E050E0EE81FF81A2
:102F80004E175F0768F4E42FF52F31970E94DC3568
:102F90003197E00FF11FE081EC934F5F5F4FEECF71
:102FA000E1E0F0E060E070E0E093490AF0934A0A63
:102FB00060934B0A70934C0A02C00E9479350E94BC
:102FC0000D340E9438340E949D3EA0C20E94973E5C
:102FD0000E947F320E940D340E9456340E947E3E31
:102FE00011F40C9450180E940D340E943635009153
:102FF000490A0E940D340E9436352091490A3091C9
:103000004A0A0E940D340E9436351091490A0E94E6
:103010000D340E9436354091490AE42F0E94C43293
:10302000FF93EF930A93EF91FF9109950E947836F1
:10303000ADE9BDE0AE0FBF1F2D933C930E947836E3
:10304000A3EABDE0AE0FBF1F1C930E947836A5E92E
:10305000BDE00E94B3320E947836ABE9BDE00E9429
:10306000BF320E947836A3E9BDE00E94BF320E94C1
:103070007836A5EABDE00E94BF320E947836A4EA05
:10308000BDE00E94BF32E1E0F0E060E070E0E0937C
:10309000490AF0934A0A60934B0A70934C0A02C0A3
:1030A0000E94E2350E940D340E943834EBC20E9427
:1030B0007F360E940D340E9456340E947E3E11F4E9
:1030C0000C94BB180E940D340E9436350091490AB9
:1030D0000E940D340E9436353091490A40914A0AC7
:1030E0000E940D340E9436350E9483360E94363588
:1030F0001091490A0E940D340E9436352091490AE8
:103100000E948A36A3EABDE00E94E032309769F45B
:103110000E9491364A933A93E0E0EA93EA85FB8570
:103120000E9495360E9423330DC0E130A0E0FA07DB
:1031300049F40A934A933A93E885F9850E949536B3
:103140000E9429330E948A36A5EABDE00E942F33EF
:103150000E948A36ABE9BDE00E942F33E1E0F0E047
:1031600060E070E0E093490AF0934A0A60934B0AEA
:1031700070934C0A02C00E949A360E940D340E943D
:1031800038346AC00E947F360E940D340E94563443
:103190000E947E3E11F40C9426190E940D340E9468
:1031A00036350091490A0E940D340E94363530911F
:1031B000490A40914A0A0E940D340E9436350E9405
:1031C00083360E9436351091490A0E940D340E94C0
:1031D00036352091490A0E948A36A3EABDE00E9452
:1031E000E032309769F40E949136EF81F885FA93C6
:1031F000EA93E0E0EA930E94A2360E9434330DC0C5
:10320000E130A0E0FA0749F40A93EE81FF81FA93D6
:10321000EA930E94A2360E943A330E948A36A5EAB7
:10322000BDE00E9440330E948A36ABE9BDE00E94B7
:103230002F33E1E0F0E060E070E0E093490AF093C2
:103240004A0A60934B0A70934C0A02C00E949A3655
:103250000E940D340E9438340E949E3E27960895A5
:103260000E947F320E940D340E9456340E947E3E9E
:1032700009F10E940D340E943635E091490AF0E0D0
:10328000F0E0A3E2B1E00E94C83BA4EABDE00E94E6
:10329000E0320E94C5350E943834E1E0F0E060E0A1
:1032A00070E0E093490AF0934A0A60934B0A7093E6
:1032B0004C0A02C00E9440350E940D340E943834EE
:1032C000089524970E947F320E940D340E94563444
:1032D0000E947E3EC9F00E947F320E94E9330E9424
:1032E000EA350E94A93A0E94C5350E943834E1E0CF
:1032F000F0E060E070E0E093490AF0934A0A6093DE
:103300004B0A70934C0A02C00E9440350E940D3453
:103310000E9438342496089528970E9456330E94BC
:1033200087320E94EE3389F1E12FF0E0A091260A66
:10333000B091270A0E94723BEA0FFB1F0E94713C6A
:10334000319766277727EA83FB836C837D8300E0D0
:103350000117C0F40E947F320E94E9336627772765
:10336000EE83FF83688779870E94A736E885F98511
:103370006A857B85EA5FFD4FFA93EA930E947D3A66
:103380000F5FE6CF0E94D63508C0A6E2BAE0BF9331
:10339000AF930E945F35AF91BF91ED93FC930E9474
:1033A0000D340E943834198108812A960895649753
:1033B0000E947F320E940D340E9456340E947E3E4D
:1033C00011F40C942B1A0E940D340E945634E88795
:1033D000F9876A877B870E940D340E945634EC83FC
:1033E000FD836E837F830E947F320E94E9336627CC
:1033F0007727E88BF98B6A8B7B8B0E947F320E9448
:10340000E9330E94B0360E94BC36D8F4E881F981D5
:103410006A817B810E94C736FF93EF93E885F98527
:103420006A857B85A889B9898A899B890E944936E2
:10343000EA5FFD4FE081AF91BF91EC930E94D036DF
:10344000E2CFEC81FD816E817F810E94C736DF0172
:10345000E0E0EC9302C00E94E2350E940D340E942D
:103460003834AFC028970E947F320E940D340E94EA
:1034700056340E947E3EA9F00E947F320E94E933BA
:103480000E94DD360E94E9330E94EA35EE81FF8119
:1034900068857985EA5FFD4FFA93EA930E949E3A28
:1034A00002C00E9440350E940D340E9438342EC064
:1034B00028970E947F320E947F320E94E9330E9447
:1034C000DD360E94E93366277727E883F9836A832C
:1034D0007B83EC81FD816E817F81EA5FFD4FFA93F2
:1034E000EA930E94A7360E948C3AA0E00E948E3B8D
:1034F0000E947E3BE093490AF0934A0A60934B0A8C
:1035000070934C0A0E940D340E9438342896089516
:1035100064970E947F320E940D340E9456340E94AC
:103520007E3E11F40C94DB1A0E947F320E94E93334
:1035300066277727E88BF98B6A8B7B8B0E940D348B
:103540000E945634E887F9876A877B87E889F9897A
:103550006A897B89EA5FFD4FFA93EA930E94A93A50
:103560000E94DD360E94E9330E94B0360E94BC36CC
:1035700008F5E885F9856A857B85AC85BD858E85EE
:103580009F850E944936EA5FFD4FFF93EF93E881E4
:10359000F9816A817B81A889B9898A899B890E947E
:1035A000363BEA5FFD4FE081AF91BF91EC930E9403
:1035B000D036DCCF02C00E9479350E940D340E94C3
:1035C0003834649608950E94973E0E947F320E948C
:1035D0000D340E9456340E947E3E11F40C943C1B24
:1035E0000E940D340E9436350091490A10914A0A12
:1035F0000E940D340E9436354091490A20E030E0A7
:103600000E947836AFE8BDE0AE0FBF1F0E94623C5B
:103610002E173F0790F40E94E436FF93EF93E42FB8
:103620000E945033EB57F34FE20FF31FE081AF914D
:10363000BF91EC932F5F3F4FE3CF0E947836AFE806
:10364000BDE0AE0FBF1F0E9492330E940D340E9456
:1036500038340E947836AFE8BDE00E94B332E1E032
:10366000F0E060E070E0E093490AF0934A0A60936A
:103670004B0A70934C0A02C00E9479350E940D34A7
:103680000E9438340E949E3E259608950E94963EE0
:103690000E947F320E940D340E9456340E947E3E6A
:1036A00011F40C94E61B0E940D340E9436350091F3
:1036B000490A10914A0A0E940D340E9436355091F1
:1036C000490A0E940D340E9436354091490A20E093
:1036D00030E0E52FF0E02E173F0778F4E42F0E944A
:1036E0005033EB57F34FE20FF31FDF010E94E43634
:1036F000E081EC932F5F3F4FECCF0E947836A1E939
:10370000BDE0AE0FBF1FE52FF0E0ED93FC930E94EC
:103710007836A4EABDE0AE0FBF1FE4E0EC930E9450
:103720007836A5E9BDE0AE0FBF1FE8EEF3E0ED93FC
:10373000FC930E947836AFE8BDE0AE0FBF1FE1E01A
:10374000F0E0ED93FC930E947836AEE8BDE00E9475
:10375000EB36F1F00E947836A8E9BDE00E94E03235
:10376000FF93EF93E081EF93E2E9F0E0FF93EF93B3
:103770000E947836A9E9BDE00E94E032AF91BF9186
:10378000EA0FFB1FE491AF91EA2BAF91BF91EC934D
:103790000E947836AAE9BDE00E94E032FF93EF93E1
:1037A000E42F0E945033EB57F34FE081AF91BF916C
:1037B000EC93E1E0F0E060E070E0E093490AF09320
:1037C0004A0A60934B0A70934C0A02C00E947935F2
:1037D0000E940D340E9438340E949D3E2696089522
:1037E0000E947F320E940D340E9456340E947E3E19
:1037F00099F0E4B7EF700E9402350E943834E1E09E
:10380000F0E060E070E0E093490AF0934A0A6093C8
:103810004B0A70934C0A02C00E947F320E940D3402
:103820000E9438340895ECE0F0E80E94713CE050CA
:10383000F048E093260AF093270A689420F820FEC7
:1038400005C00E9470320E941C36F9CF0895EFEF38
:10385000E3B9E0E0E2B9E8BBEFEFE7BBE091650078
:10386000E260E09365000895E1B1E095E09306021F
:10387000089B02C0D89801C0D89A099B02C0D99869
:1038800001C0D99A0A9B02C0DA9801C0DA9A0B9B50
:1038900002C0DB9801C0DB9A0C9B02C0DC9801C01F
:1038A000DC9A0D9B02C0DD9801C0DD9A0E9B02C020
:1038B000DE9801C0DE9A0F9B02C0DF9801C0DF9A3C
:1038C000E0916300E270E23069F4E8E0F2E0FF9337
:1038D000EF93E081AE2FEAE9F0E0E491EA23AF91C3
:1038E000BF910CC0E8E0F2E0FF93EF93E081AE2FD0
:1038F000E2E9F0E0E491EA2BAF91BF91EC93E09123
:103900000702E8BBC09B02C0AF9A01C0AF98C19B41
:1039100002C0AE9A01C0AE98C29B02C0AD9A01C06F
:10392000AD98C39B02C0AC9A01C0AC98C49B02C0C6
:10393000AB9A01C0AB98C59B02C0AA9A01C0AA98D5
:10394000C69B02C0A99A01C0A998C79B02C0A89AA9
:1039500001C0A89808950A921A926A937A93AA933A
:10396000BA93EA93FA93EFB7EA930A93E6E0E2BFD9
:10397000E091810CF091820C6091830C7091840C29
:10398000EF5FFF4F6F4F7F4FE093810CF093820CFE
:103990006093830C7093840CA89500E0013010F0C4
:1039A0000C944B1D0E94AC32A5E9BDE0AE0FBF1FC9
:1039B0000E94623C309711F40C94491D0E94AC3275
:1039C000A5E9BDE0AE0FBF1F0E94623C3197ED93A9
:1039D000FC93309711F00C94491D0E94AC32A4EA7C
:1039E000BDE00E94E032E230A0E0FA0749F40E9414
:1039F000AC32A4EABDE0AE0FBF1FE5E0EC9349C0D6
:103A0000E330A0E0FA0739F40E94AC32A4EABDE04A
:103A10000E94BF323EC0E130A0E0FA0749F40E94A4
:103A2000AC32A4EABDE0AE0FBF1FE6E0EC9331C0BC
:103A3000E430A0E0FA0769F50E94AC32A4EABDE0E8
:103A40000E94BA32A5EABDE00E94BA32AEE8BDE0FB
:103A50000E94EB36F1F00E94AC32A8E9BDE00E9472
:103A6000E032FF93EF93E081EF93EAE9F0E0FF9318
:103A7000EF930E94AC32A9E9BDE00E94E032AF9121
:103A8000BF91EA0FFB1FE491AF91EA23AF91BF9181
:103A9000EC930F5F83CF0991E991EFBFF991E99121
:103AA000B991A991799169911990099018950E94FD
:103AB000F036E0919C000E945D320DD00E94FE36EF
:103AC00018950E94F036E5E8FCE0FA93EA934DD0B1
:103AD0000E94FE3618950E940C37E2E0EA17C0F10A
:103AE0000E940C37A230E9F0EA81A0910002EA17A7
:103AF00039F0A881B981A25EBE4FAC91A03051F0DF
:103B00000E9412370E9417370E941E37A15EBE4FD7
:103B1000E2E005C0A881B981A15EBE4FE3E0EC936D
:103B200017C00E942637E930A1E0FA0770F40E941E
:103B30002637A881B981EA0FFB1FAA81A0830E94C2
:103B400026373196ED93FC9303C00E942D37EC93FA
:103B5000A881B981A15FBE4FEC91F0E0A881B98145
:103B6000A05FBE4FED93FC93A5C00E940C37A4301C
:103B700011F00C94201E0E942637FF93EF93A8812A
:103B8000B981A45FBE4F0E94623CAF91BF91AE1756
:103B9000BF07B0F4A881B9810E943337FF93EF9338
:103BA0000E942637A881B981AE0FBF1FEC91AF915B
:103BB000BF91EC930E9426373196ED93FC9340C061
:103BC0000E943837B1F00E943F37FF93EF93E081B6
:103BD000EF93EAE9F0E0FF93EF930E944637AF914D
:103BE000BF91EA0FFB1FE491AF91EA23AF91BF9120
:103BF000EC93A881B981AA5EBE4FAC91E0E0EA17D0
:103C000090F4A881B981A85EBE4F0E94623CA88151
:103C1000B981A05FBE4FED93FC93A881B981A15EED
:103C2000BE4FE1E002C00E942D37EC93A881B9811C
:103C3000A65FBE4FE0E0F0E0ED93FC930E944D37AD
:103C4000229608950E9412371196E2E0EC93A88123
:103C5000B981A45FBE4FE2E0F0E0ED93FC93A88150
:103C6000B9810E945337A881B9810E945837A88131
:103C7000B9810E9417370E943837B1F00E943F3750
:103C8000FF93EF93E081EF93E2E9F0E0FF93EF938E
:103C90000E944637AF91BF91EA0FFB1FE491AF91AD
:103CA000EA2BAF91BF91EC930E941E370E943337ED
:103CB000AA81A083239608951A930A93EB850E9404
:103CC0005F37E0910002EC93AA81BB811296E0E09D
:103CD000EC93EA85AA81BB811396EC93E885AA81CF
:103CE000BB811496EC93E985F070AA81BB8115968F
:103CF000EC93EF81AA81BB811696EC93ED81AA81AA
:103D0000BB811796EC93EE81F070AA81BB81189667
:103D1000EC93EC81AA81BB811996EC93EAE0F0E088
:103D20000E946437AA81BB811A96EC93AA81BB8159
:103D30001B960E947137ECE0F0E00E947737AA8171
:103D4000BB810E945837AA81BB810E9417370E940D
:103D50007C37B1F00E948337FF93EF93E081EF93BC
:103D6000E2E9F0E0FF93EF930E948A37AF91BF91B1
:103D7000EA0FFB1FE491AF91EA2BAF91BF91EC9357
:103D80000E949137AA81BB810E943337AB85A08303
:103D9000198108812C96089522970E94993EEE85FC
:103DA000AD81BE81EC931196E0910002EC93AD8160
:103DB000BE811296E1E0EC93ED85AD81BE81139654
:103DC000EC93EB85AD81BE811496EC93EC85F0709D
:103DD000AD81BE811596EC93EF81AD81BE811696C3
:103DE000EC93EA85F0E03097C1F4E6E0F2E0A885D4
:103DF000B985EA0FFB1FEB83FC8300E0EF810E1710
:103E000058F40E949737FF93EF930E949F37AF912A
:103E1000BF91EC930F5FF2CF66C0E130A0E0FA07EC
:103E2000D1F4E885F985EB83FC8300E0EF810E1780
:103E300088F40E949737FF93EF93AB81BC81119672
:103E4000AB83BC8311970E94963CAF91BF91EC93DA
:103E50000F5FECCF48C0E230A0E0FA07D9F4E88564
:103E6000F985E050F048EB83FC8300E0EF810E170A
:103E700080F40E94A537AD81BE81AE0FBF1FEB81DC
:103E8000FC813196EB83FC833197E491EC930F5FD7
:103E9000EDCF29C0E330A0E0FA07A1F4E885F98569
:103EA000EB83FC8300E0EF810E1758F40E949737F4
:103EB000FF93EF930E949F37AF91BF91EC930F5FF9
:103EC000F2CF11C0E430A0E0FA0769F4E885F98583
:103ED000309729F4AD81BE8117964C9204C0E13031
:103EE000A0E0FA0701F40E94A937FA93EA93EF8160
:103EF000F885FA93EA93E0D41E2F2F2F0E94A9375A
:103F0000AD81BE81AE0FBF1FE22FF0700E94AD37B2
:103F10003896AD81BE81AE0FBF1F1C93EF81F0E0DC
:103F20003996AD81BE81A45FBE4FED93FC93AD8108
:103F3000BE810E945337AD81BE810E945837AD814A
:103F4000BE810E941737AD81BE810E94B137D1F08A
:103F5000AD81BE810E94B637FF93EF93E081EF936E
:103F6000E2E9F0E0FF93EF93AD81BE810E94BB37A1
:103F7000AF91BF91EA0FFB1FE491AF91EA2BAF9194
:103F8000BF91EC930E949137AD81BE810E9433377F
:103F9000AE85A0830E94A03E2F96089522970A9393
:103FA000E885F0E03097D1F4E6E0F2E0AE81BF8141
:103FB000EA0FFB1FE983FA8300E0ED810E1768F436
:103FC0000E94C037FF93EF930E94A5370E94C73726
:103FD000AF91BF91EC930F5FF0CF5DC0E130A0E0F7
:103FE000FA07B9F4EE81FF81E983FA8300E0ED81FD
:103FF0000E1770F40E94C037FF93EF930E94A5370D
:104000000E94C737AF91BF910E94B53C0F5FEFCFC1
:1040100042C0E230A0E0FA0789F4AE81BF81A0502F
:10402000B048FD01EF2FF0E0FA93EA93ED81FE81B5
:104030003796FA93EA930E94107E2DC0E330A0E0F9
:10404000FA07B1F4EE81FF81E983FA8300E0ED81A4
:104050000E1768F40E94C037FF93EF930E94A537B4
:104060000E94C737AF91BF91EC930F5FF0CF13C0A1
:10407000E430A0E0FA0779F4EE81FF81309739F45B
:10408000AB81BC811796EC91E093010204C0E13052
:10409000A0E0FA0701F40881299608951A930A937B
:1040A000E9850E945F37E3E0EC93E885F070AA8130
:1040B000BB811296EC93EF81AA81BB811396EC939E
:1040C000AA81BB811496E0E0EC93EC81AA81BB81CC
:1040D0001596EC93E6E0F0E00E946437AA81BB817C
:1040E0001696EC93AA81BB8117960E947137E8E07F
:1040F000F0E00E947737AA81BB810E945837AA81DD
:10410000BB810E941737E985AA81BB81A55EBE4F9E
:10411000EC93ED81FE81AA81BB81A45EBE4FED933D
:10412000FC930E947C37B1F00E948337FF93EF939A
:10413000E081EF93E2E9F0E0FF93EF930E948A378A
:10414000AF91BF91EA0FFB1FE491AF91EA2BAF91C2
:10415000BF91EC930E949137AA81BB810E943337B3
:10416000A985A083198108812A9608950E94983E06
:10417000EB85AC81BD81EC931196E6E0EC93EA858A
:10418000F070AC81BD811296EC93E985AC81BD8164
:104190001396EC9300E0EE810E1730F5E02FEE0F52
:1041A0001E2FE12FF0E03496AC81BD81EA0FFB1F9A
:1041B000FF93EF930E94CD370E94D437AF91BF9108
:1041C000EC93E12FF0E03596AC81BD81EA0FFB1F47
:1041D000FF93EF930E94CD37EA5FFD4FE081AF91EF
:1041E000BF91EC930F5FD7CF0E94D937FA93EA9330
:1041F000EE81FF81FA93EA935FD32E2F3F2F0E9427
:10420000D937AC81BD81AE0FBF1FE32FF070EC93A7
:104210000E94DF373596AC81BD81AE0FBF1F2C9356
:104220000E94DF373696AC81BD81A45FBE4FED930F
:10423000FC93AC81BD810E945337AC81BD810E944B
:104240005837AC81BD810E941737EB85AC81BD81A9
:10425000A55EBE4FEC93AC81BD810E94B137D1F019
:10426000AC81BD810E94B637FF93EF93E081EF935D
:10427000E2E9F0E0FF93EF93AC81BD810E94BB3790
:10428000AF91BF91EA0FFB1FE491AF91EA2BAF9181
:10429000BF91EC930E949137AC81BD810E9433376E
:1042A000AB85A0830E949F3E2C960895289781E0BD
:1042B000A0E0B0E0E8E5F3E00E94A43E0E94963E54
:1042C0000E944D37AE85BF85A15EBE4FE0E0EC9306
:1042D000AE85BF85A25EBE4F0E94E43711F00C94FC
:1042E000F9210E94E83711F00C94C6210E94ED37A5
:1042F00011F00C94C5210E94FD37FF93EF930E94AB
:104300000438AF91BF91EA0FFB1F0E2F1F2FAE8510
:10431000BF8512960E94E43741F5AE85BF85189699
:10432000EC91FE2FE0E0FF93EF93AE85BF851796EB
:10433000EC91F0E0AF91BF91EA0FFB1F2E2F3F2FC2
:104340000E940A38A681AA933A932A93EA89FB89A4
:104350000E941138ED89FE89A185AA93EE89FF8913
:10436000FA93EA930E94CC1E10C0E130A0E0FA0755
:1043700061F4EE85FF850E9411380E9416380E9474
:104380000A38FA93EA930E94221E32C0E130A0E07C
:10439000FA0711F50E94ED3731F4AE85BF8512960C
:1043A000AC91A13009F013C00E94FD37FF93EF9349
:1043B0000E940438AF91BF91EA0FFB1F0E2F1F2FF1
:1043C000EE85FF850E9411380E94163802C00E94B7
:1043D00020380E9427380CC0E230A0E0FA0741F4F0
:1043E0000E942E38A23011F00E9420380E942738F7
:1043F00015C2E130A0E0FA0711F00C940A240E94E3
:10440000E83711F00C94A623AE85BF85EC91A091FE
:104410000002EA1711F00C94A5230E94ED3711F069
:104420000C94A5230E943338FE2FE0E0FF93EF9316
:10443000AE85BF851396EC91F0E0AF91BF91AE0FC2
:10444000BF1FE2E0F0E00E94C83BEF83AE85BF856E
:104450001196EC91F0E0E330A0E0FA07F1F50E944C
:104460003838FF93EF930E943F38AF91BF910E947D
:104470004538AE85BF851296EC93E0E0EA87EB877E
:104480000E944C38D8F40E9453380E945A38FF9347
:10449000EF930E9462380E94D437AF91BF910E947F
:1044A0006938FF93EF930E946238EA5FFD4FE08125
:1044B000AF91BF91EC930E947238E2CF0E9478389E
:1044C0000E947E380E948938AE85BF85A45FBE4FAA
:1044D000ED93FC93E1E0EE83FFC0E430A0E0FA0747
:1044E00011F00C94D9220E943838FF93EF930E9468
:1044F0003F38AF91BF910E944538AE85BF85129677
:10450000EC93E0E0EA87EB87EC85FD850E94A0381C
:1045100010F00C94CA220E94A7380E945A38FF93C8
:10452000EF930E9462383396EA5FFD4FE081AF91CE
:10453000BF910E946938FF93EF930E9462383296D0
:10454000EA5FFD4FE081AF91BF91EC93E885F9857B
:104550003596AE85BF85EA0FFB1FFF93EF930E9450
:1045600062380E94D437AF91BF91EC93E885F9850A
:104570003696AE85BF85EA0FFB1FFF93EF930E942F
:104580006238EA5FFD4FE081AF91BF91EC930E94EA
:104590007238BACF0E9478380E947E380E948938DB
:1045A000AE85BF85A45FBE4FED93FC93E1E0EE8343
:1045B00093C0E630A0E0FA07E9F4EF81F0E0EA5FAB
:1045C000FD4FFF93EF93AE85BF851596EC91AF91AC
:1045D000BF910E94AD373196EA5FFD4FFF93EF9395
:1045E000AE85BF851496EC91AF91BF91EC930E947C
:1045F000AE3872C0E031A0E0FA0711F00C946C23E1
:10460000AE85BF851696EC91F0E00E94793BEC8771
:10461000FD87E0E0EA87EB870E944C3810F00C94AD
:1046200055230E94A7380E946238EA5FFD4FFF932E
:10463000EF93E885F9853A960E94B938AF91BF911A
:104640000E94AD370E94BF38FF93EF93E885F9854C
:1046500039960E94B938AF91BF910E94AD37A885B5
:10466000B985EA0FFB1F3296EA5FFD4FFF93EF9388
:10467000E885F98538960E94B938AF91BF910E94BC
:10468000AD37A885B985EA0FFB1F3396EA5FFD4F6A
:10469000FF93EF93E885F98537960E94B938AF917B
:1046A000BF91EC930E947238B7CFE6E0F0E0FA9346
:1046B000EA93E889F989FA93EA93FED04E2F5F2FA7
:1046C000E52FF070AE85BF851696EC93AE85BF855D
:1046D00017964C930E94AE38EE81E030B1F1AE8572
:1046E000BF850E945337AE85BF850E945837AE857F
:1046F000BF850E941737AE85BF850E94B137D1F0C4
:10470000AE85BF850E94B637FF93EF93E081EF93AC
:10471000E2E9F0E0FF93EF93AE85BF850E94BB37DF
:10472000AF91BF91EA0FFB1FE491AF91EA2BAF91DC
:10473000BF91EC930E949137AE85BF85AB5EBE4FB3
:10474000AC91BB27E0910002EC9363C0E130A0E0A4
:10475000FA0711F00C94F2230E94ED3769F4AE854C
:10476000BF85EC91EF930E94C738AF91EA1721F40F
:104770000E942E38A33009F031C0E0E0EA87EB87D1
:104780000E943338F0E00E94A03828F50E94533888
:104790000E94CD380E94BF38FF93EF93E885F985DA
:1047A00033960E94B938AF91BF91EC930E94CD38F7
:1047B000A885B985EA0FFB1FEA5FFD4FFF93EF93D2
:1047C000E885F98534960E94B938AF91BF91EC9392
:1047D0000E947238D5CF0E94D43802C00E94DA38C5
:1047E000EC9317C0E230A0E0FA0799F40E94ED378D
:1047F00049F4AE85BF85EC91EF930E94C738AF9125
:10480000EA1709F003C00E94D43802C00E94DA38C7
:10481000EC9304C0E230A0E0FA0701F40E949D3E50
:1048200060960895EA81A881B981AE5EBE4FEC938F
:10483000F0E0309739F4A881B981A15FBE4FEAE07A
:10484000EC9338C0E130A0E0FA0739F4A881B981CF
:10485000A15FBE4FE5E0EC932DC0E230A0E0FA0787
:1048600039F4A881B981A15FBE4FE3E0EC9322C087
:10487000E330A0E0FA0719F40E94E0381BC0E430EE
:10488000A0E0FA0719F40E94E03814C0E530A0E077
:10489000FA0719F40E94E0380DC0E630A0E0FA07EC
:1048A00019F40E94E03806C0E730A0E0FA0711F4DE
:1048B0000E94E038239608950E94983E0FEF1FEF64
:1048C00020E030E0EE81FF812E173F0728F5E02F32
:1048D000F12FFE2FE0E0FF93EF93EAE5F3E0FF9383
:1048E000EF93E12FF070FF93EF93E22FF32FAC8162
:1048F000BD810E94E032AF91BF91EA27FB27AF91C3
:10490000BF910E94E738AF91BF91EA27FB270E2F96
:104910001F2F2F5F3F4FD6CFE02FF12F32C00E94C5
:10492000983E0FEF1FEF20E030E0EE81FF812E1761
:104930003F0728F5E02FF12FFE2FE0E0FF93EF93E4
:10494000EAE5F3E0FF93EF93E12FF070FF93EF932D
:10495000E22FF32FAC81BD810E94F432AF91BF9161
:10496000EA27FB27AF91BF910E94E738AF91BF9133
:10497000EA27FB270E2F1F2F2F5F3F4FD6CFE02FA9
:10498000F12F0E949F3E28960895FFFFFFFFFFFF33
:10499000FFFFFFFFFFFFFFFFFFFFFFFFFFFFFFFF27
:1049A000FFFFFFFFFFFFFFFFFFFFFFFFFFFFFFFF17
:1049B000FFFFFFFFFFFFFFFFFFFFFFFFFFFFFFFF07
:1049C000FFFFFFFFFFFFFFFFFFFFFFFFFFFFFFFFF7
:105000005F9BFECFACB108955D9BFECFA881ACB98C
:1050100021960895A881B9810E94623C309731F0B1
:105020000E94EE383197AA81A08304C0EA81EA93F6
:105030000E940428239608950E94F438A885E5E08C
:10504000EA1708F4E887AAE5B5E0E885F0E00E94F1
:10505000723BEA0FFB1F0E94753CA985BA858B85C0
:105060009C850E94853DE987FA876B877C8700E0F5
:10507000E0E0F0E060E87FE3EA83FB836C837D831C
:10508000EA81FB816C817D81A985BA858B859C85B0
:105090000E94463E80F0AA81BB818C819D81E0E028
:1050A000F0E060E271E40E94D33DEA83FB836C830D
:1050B0007D830F5FE5CF003029F40E94F838E0E3EC
:1050C000EC932AC0E02F0150E03031F1AA81BB817E
:1050D0008C819D810E94FF38EA83FB836C837D83F2
:1050E000A985BA858B859C850E940F390E94F83866
:1050F0000E941539AA81BB818C819D81FF2766277B
:1051000077270E94473D0E94D33DA985BA858B85AC
:105110009C850E941A39D6CFE885E03019F40E94A8
:1051200023392CC00E94F838EEE2EC93E885E15078
:10513000E887EF5F09F1A985BA858B859C85E0E05A
:10514000F0E060E271E40E94D33DE987FA876B8763
:105150007C870E94143D1E2F0E94F8380E9415394A
:10516000A985BA858B859C85FF27662777270E94AE
:10517000473D0E941A39DACF0E94233919810881EC
:105180002D96089524970E94993EE0E0F0E060E8B3
:105190007FE3EB83FC836D837E83AA85E5E0EA17DA
:1051A00008F4EA870A85E02F0150E03019F00E94E8
:1051B0002839F9CFEB85FC856D857E850E947E3E82
:1051C00021F420E00E9428393AC02A850E9437390C
:1051D00009F010F40C94F6280E9428390E943739FF
:1051E00020F00E9442392F5FF9CF15C00E94373955
:1051F00080F4AB85BC858D859E85E0E0F0E060E2C3
:1052000071E40E94D33DEB87FC876D877E87215038
:10521000EDCF0E942839EB85FC856D857E85A0E069
:10522000B0E080E09FE30E94853DEB87FC876D87BF
:105230007E870E94373918F00E9442392F5F00E0C4
:10524000EA85E017A0F1AB81BC818D819E810E942F
:10525000FF38EB83FC836D837E83AB85BC858D85B6
:105260009E850E940F390E9451390E941539FF27EF
:10527000662777270E94473DAB81BC818D819E8147
:105280000E94D33DAB85BC858D859E850E94803C68
:105290000E947E3DEB87FC876D877E87E02F0F5F46
:1052A000E03071F60E945139EEE2EC93C9CF0E94D2
:1052B0005839A985A08320302CF40E945139EDE2A1
:1052C000EC932195E9E0E21764F40E945839FF93CA
:1052D000EF93A22FEAE00E94033CE05DAF91BF9103
:1052E000EC930E945839FF93EF93A22FEAE00E94BB
:1052F000333CE05DAF91BF91EC93AF81B885E0E0C6
:10530000EC930E94A03E2F9608951B7FE989EA93B3
:10531000EBA1FCA1FA93EA937DDE403009F04A95B7
:1053200008956C970E94963E00E0EEA1FFA1319691
:10533000EEA3FFA33197E4913E2FE03011F40C94DB
:10534000BC2BE02FF0E0309739F4353211F401E056
:1053500002C00E945F390FC2E130A0E0FA07C9F431
:10536000353221F40E945F3900E005C202E0E0E03E
:10537000E98B10E03D3211F411E0FDC13B3219F42C
:10538000EBE2E98BF8C1303219F4E0E2E98BF3C1CA
:1053900004C0E230A0E0FA0739F440E003E0303323
:1053A00011F41068E8C104C0E330A0E0FA0789F402
:1053B000303310F03A3308F006C00E946639E32F0C
:1053C000E0534E0FD8C150E03E3211F404E0D3C197
:1053D00011C0E430A0E0FA0799F4303310F03A330A
:1053E00008F008C010620E946C395E2FE32FE05372
:1053F0005E0FC1C13C3619F4126005E0BCC106C0A5
:10540000E530A0E0FA0711F00C94BB2BE32FF0E09D
:10541000E336A0E0FA0731F40E947139EC910E9462
:105420007839A8C1E534A0E0FA0721F0E536A0E01C
:10543000FA0709F404C0E636A0E0FA07F1F5FE0128
:105440007296EE83FF830E9471390E94663CE88762
:10545000F9876A877B87DF01CB010E94823E24F0B7
:10546000A989AB3229F00EC00E947F39EDE2E98BA9
:1054700017FF04C0E9890E94783904C00E948A3964
:10548000A989A08315FF55E0363649F40E94913969
:10549000EB85FC85FA93EA930E941C2809C00E94C0
:1054A00091393A93EC85FD85FA93EA930E94C228DC
:1054B000FE0172960E94993922C0E337A0E0FA07F4
:1054C00039F40E9471390E94623C0E94993910C0DF
:1054D000E037A0E0FA07C1F40E9471390E94623CF3
:1054E000EE83FF83FA93EA930E94B33A0E2F18607B
:1054F0001F77503011F0501708F001C0052F50E011
:10550000E0E0E88B20E089C0E436A0E0FA0721F073
:10551000E936A0E0FA0711F4146004C0E537A0E012
:10552000FA07C1F4EAE0E88B11FF0AC0E0E0FAEC08
:105530006AE97BE3EC87FD876E877F870AE02DC0F1
:10554000E0E1F7E260E070E0EC87FD876E877F873F
:1055500005E023C0E835A0E0FA0711F4186006C0A2
:10556000E837A0E0FA0711F00C94BA2BE0E1E88BE1
:1055700011FF0AC0E0E0F0E060E070E1EC87FD8739
:105580006E877F8708E009C0E0E0F0E160E070E04E
:10559000EC87FD876E877F8704E0503011F01F771E
:1055A00001C051E011FF09C00E9471390E94663CA0
:1055B000E887F9876A877B8713C012FF07C00E94BC
:1055C00071390E94623C0E94843B06C00E9471397E
:1055D0000E94623C66277727E887F9876A877B877E
:1055E00012FF1AC0A885B9858A859B850E94823ED4
:1055F00064F4E885F9856A857B850E944F3BE887DE
:10560000F9876A877B87EDE2E98BE989E03019F059
:105610000F5F5F5F01C01B7F252F10FD14C00417B3
:1056200010F4241708F00FC017FF08C012FF04C0C1
:105630001B7F3989015001C030E301C030E20E9474
:105640005F394150ECCF051778F4106112FF04C0A8
:105650000E94852901505150E0E30E947839403082
:1056600009F041505150EFCF202FE889E030D1F4BC
:105670002030B9F013FF04C00E948A39E49105C0BC
:10568000AE81BF81ED91AE83BF83EA93EBA1FCA114
:10569000FA93EA930E940A28403009F041502150C1
:1056A000E7CF5FC0EC85FD856E857F85A885B985D0
:1056B0008A859B850E94083C3E2FE9E0E31730F481
:1056C00013FF02C0395C01C0395A01C0305D14FDBE
:1056D00022C0E0E3E31760F0AC85BD858E859F8531
:1056E000A130E0E0BE07E0E08E07E0E09E0709F4AD
:1056F0000DC0521710F030E309C0421710F010FF30
:1057000001C00EC030E217FF06C030E3106112FF87
:1057100002C00E9485290E945F39403009F0415043
:105720002150EC85FD856E857F85A885B9858A85A4
:105730009B850E943F3CE887F9876A877B87E889D9
:10574000F0E0AC85BD858E859F85662777270E9412
:10575000083CEC87FD876E877F870E947E3E09F0BC
:10576000A1CF10FF07C0403029F04150E0E20E9475
:105770007839F9CF00E0D9CD0E949D3EA8960895D2
:10578000FF92F82E0E94A1390E949129AA81BB8123
:10579000E0E0EC933CC10A93AB81BC81EC910E2F0D
:1057A000E03019F0E0E0EC9312C0A981BA810E94C8
:1057B000623C309749F00E94623CE0810E2FE0305D
:1057C00011F00E94EE3803C00E9400280E2FE02F37
:1057D00008812596089527970E94963EE0E0EB8782
:1057E000EC87E989FA893196E98BFA8B3197E49154
:1057F0002E2FE03011F40C94FC2C0E94C03961F083
:105800000E94C5392E2FE03019F00E94C03909F4EA
:1058100001C0F6CF2C87EFC0253211F00C94F12C8B
:1058200040E00E94CF39203318F0E9E3E21708F492
:1058300006C00E946639E22FE0534E0FF2CF2030AF
:1058400009F4DAC00E94C5393E2F0E94D539D1F73C
:10585000303009F4CAC03C87403009F44FEF50E0C3
:10586000E22FF0E0E336A0E0FA0741F40E94DA39D3
:105870000E94C539A02FB12FEC93AFC0E337A0E051
:10588000FA07E9F40E94DA39E42F4150E03091F050
:105890000E94C5392E2FE03019F00E94C03909F05E
:1058A00009C01F930F930F5F1F4FE22FAF91BF915E
:1058B000EC93EACFA02FB12FE0E0EC938EC0EC3652
:1058C000A0E0FA0719F451E00E94CF39E1E0EA873D
:1058D000E22FF0E0E436A0E0FA0721F0E936A0E09C
:1058E000FA0719F4E0E0EA8704C0E537A0E0FA0718
:1058F00011F43AE00DC0E837A0E0FA0711F430E106
:1059000007C0E532A0E0FA0709F46BC0EB8575C06B
:10591000E0E0EE83EF83E887E987E42F4150E03051
:10592000B9F10E94C5392E2FAE2FE0E2EA17B8F484
:10593000EA85E03039F42D3219F4EFEFEA87EDCF44
:10594000E1E0EA87203358F0213610F0275505C0F2
:10595000213410F0275301C02053231710F02C8757
:1059600017C0E32FF0E0AE81BF8188859985662757
:1059700077270E94D03BDF01CB01E22FF0E06627C2
:1059800077270E94363BEE83FF8368877987C5CFF0
:10599000EA85F0E0E7FDFFEFAE81BF81888599855C
:1059A0000E94843B0E94D03BEE83FF836887798707
:1059B000503059F00E94DA39EE81FF81688579858F
:1059C000A02FB12F0E946C3C08C00E94DA39EE81F2
:1059D000FF81A02FB12FED93FC93EB85EF5FEB8759
:1059E0000AC00E94C539E21731F0EB85E03011F4AE
:1059F000EFEF03C001C0F5CEEB850E949D3E63969C
:105A00000895FF92F82E0E94A1390E94EB2B198174
:105A100008812496FF900895E991F991699179910F
:105A200030976040704042F4E095F0956095709535
:105A300000243196601D701D089566277727A9916F
:105A4000B99189919991E1E0FF27AE1BBF0B860BBD
:105A5000970B18F03296671FF8CF6695F795E79584
:105A60000895E991F991699179917F770895249743
:105A7000EC81FD816E817F810E947E3E29F4E0E011
:105A8000F0E060E070E0E7C1EC81FD816E817F8134
:105A9000A885B9858A859B850E94053EE883F983A0
:105AA0006A837B830E947E3E29F4E0E0F0E060E0C0
:105AB00070E0D1C1A881B9818A819B810E94863E14
:105AC0004CF4E881F9816A817B810E947B3C0E94D1
:105AD000233B08C0E881F9816A817B810E947B3C7D
:105AE0000E94293BE883F9836A837B83AC81BD8173
:105AF0008E819F810E94D33DA885B9858A859B852B
:105B00000E94803C0E947E3DA6C10E94F438AE8176
:105B1000BF81888599850E94863E2CF0EFEFFFEFCC
:105B20006FE77FEF8AC0EE81FF81688579850E94EB
:105B30007B3CEDB7FEB73197FA93EA931F930F932F
:105B40000E94CA3C0F911F91EE83FF83688779877B
:105B5000AE81BF8188859985E3EFF4E065E37FE35B
:105B60000E94463E60F4EE81FF81688579850E943F
:105B7000853DEE83FF836887798701501040AE81B1
:105B8000BF81888599850E94E3397F936F93FF9346
:105B9000EF93EE81FF8168857985A0E0B0E080E831
:105BA0009FE30E94853DAF91BF918F919F910E948D
:105BB000053E0E94EC39A6E2B2E485E69FE30E942E
:105BC000D33DDF01CB01EEE4F1E164E570E40E9436
:105BD000803C0E947E3DAE81BF81888599850E9470
:105BE000D33D7F936F93FF93EF93AA81BB818C8109
:105BF0009D81EDE4F1E164ED7FE30E94803C0E9431
:105C00007E3DAF91BF918F919F910E94053E7F9302
:105C10006F93FF93EF93E02FF12FA8E1B2E781E3B9
:105C20009FE30E94843B0E94473D0E94D33DAF9179
:105C3000BF918F919F910E94853D198108812A967D
:105C4000089528971A930A93AA85BB858C859D850C
:105C5000E0E5FCEA6EEA72EC0E94463E28F4E0E0E1
:105C6000F0E060E070E095C0EA85FB856C857D859D
:105C70000E947E3E29F4E0E0F0E060E87FE389C026
:105C8000AA85BB858C859D85E8E1F2E761EB72E42E
:105C90000E94463E09F010F40C94532EEFEFFFEFF4
:105CA0006FE77FE776C0AA85BB858C859D85EBE392
:105CB000FAEA68EB7FE30E94D33DEA87FB876C87B3
:105CC0007D870E947B3C0E94233B0E94143D0E2F47
:105CD0001F2FE02FF12FAA85BB858C859D850E9403
:105CE000843B0E94473D0E94AF350E94803C0E9449
:105CF0007E3D0E94EC39ADE6BCE48CE69DE30E945B
:105D0000D33DA6EAB3EE86EE90E40E94853DAE81D7
:105D1000BF81888599850E94D33DEE83FF83688784
:105D20007987EA81FB816C817D81A8E2BDE886EA02
:105D300091E40E94853DEA83FB836C837D83EE8141
:105D4000FF8168857985AA81BB818C819D810E94B4
:105D5000853DA3EFB4E085EB9FE30E94D33D7F93A5
:105D60006F93FF93EF93AE81BF8188859985EA8118
:105D7000FB816C817D810E947E3DAF91BF918F91AF
:105D80009F910E94053E0E947B3C1A930A930E94B9
:105D9000DD3C198108812E9608952497E885F985C0
:105DA0006A857B850E947E3E29F4E0E0F0E060E0B9
:105DB00070E051C0A885B9858A859B850E94863E82
:105DC0009CF4EC81FD816E817F810E947E3E29F4EE
:105DD000E0E0F0E060E87FE33EC0E885F9856A85B1
:105DE0007B850E94FB3937C0EC81FD816E817F810C
:105DF000DE010E94143D0E946C3CE881F9816A81B9
:105E00007B810E94473DDF01CB01EC81FD816E81EA
:105E10007F810E948C3E29F0E0E0F0E060E070E0DD
:105E20001AC0E885F9856A857B850E94EB3C0E9453
:105E3000FB39E887F9876A877B87E881E17029F475
:105E4000E885F9856A857B8506C0E885F9856A85D8
:105E50007B850E94EB3C2C96089524970A9300E0E2
:105E6000AD81BE818F819885E3E8F9EF62E27EE340
:105E70000E94D33DED83FE836F8378870E947B3C35
:105E80000E94233BAD81BE818F8198850E94093A93
:105E9000AD81BE818F819885E0E0F0E060E07FE336
:105EA0000E94463E09F010F40C94592F0E94093AC2
:105EB00001E0AD81BE818F819885E0E0F0E060E88F
:105EC0007EE30E94463E09F010F40C94712FE0E04E
:105ED000F0E060E07FE30E947E3DED83FE836F8310
:105EE0007887003011F00E94123A0E941D3AE9832F
:105EF000FA836B837C83A1EBB4EC86E292E40E948C
:105F0000D33DDF01CB01EDE1F5EE6DE272E40E94DD
:105F1000803C0E947E3DA981BA818B819C810E9438
:105F2000D33DACE4B3E584E091E40E94853DAD81CE
:105F3000BE818F8198850E94D33D7F936F93FF939D
:105F4000EF93E981FA816B817C81A1E1BDEE8EED59
:105F50009FE30E94853DA981BA818B819C810E942B
:105F6000D33DAEE5BBE788EA9FE30E94853DAF9154
:105F7000BF918F919F910E94053E34C1A881B98144
:105F80008A819B81EBEDFFE069EC7FE30E947E3D1F
:105F90000E947B3C0E942D2F6AC12497EC81FD81D9
:105FA0006E817F810E947B3C0E94BE2FE883F98333
:105FB0006A837B830E947E3E89F4AC81BD818E81A1
:105FC0009F810E94863E2CF4EFEFFFEF6FE77FE7A3
:105FD0004BC0EFEFFFEF6FE77FEF46C0EC81FD8135
:105FE0006E817F810E947B3C0E942D2FDF01CB01BF
:105FF000E881F9816A817B810E94053E35C0249742
:10600000EC81FD816E817F81AC81BD818E819F811C
:106010000E94D33DE883F9836A837B83A5E6B0EDD4
:106020008BEC90E40E94283AAC81BD818E819F81E7
:106030000E94D33D7F936F93FF93EF93E881F981A3
:106040006A817B81A0E0BDE689E291E40E94853D02
:10605000A881B9818A819B810E94283AAF91BF9122
:106060008F919F910E94053E28960895A881B9813D
:106070008A819B81EDECF3E164ED7EE30E94463E74
:1060800048F4E881F9816A817B810E947B3C0E940F
:10609000FF2FEDC0A881B9818A819B81EAE7F2E8F0
:1060A0006AE170E40E94463E09F010F40C946530F9
:1060B000E881F9816A817B81A0E0B0E080E89FE31C
:1060C0000E94313A0E94373AD2C0A881B9818A81B0
:1060D0009B810E94E3397F936F93FF93EF93E88155
:1060E000F9816A817B81A0E0B0E080E89FE30E94B3
:1060F000853DAF91BF918F919F910E94313AABED59
:10610000BFE089E49FE30E94853DB1C024970A93D4
:1061100000E0AD81BE818F819885E0E0F0E060E82D
:106120007FEB0E94463E58F0E0E0F0E060E87FE35D
:106130000E94463E19F010F00C949F3005C0EFEF1E
:10614000FFEF6FE77FE74EC0AD81BE818F819885FD
:106150000E94823E1CF40E94123A01E00E941D3A05
:10616000A0E0B0E080E89FE30E94803C0E947E3D7A
:106170000E947B3C0E94BE3AE983FA836B837C8356
:10618000AD81BE818F819885E3EFF4E065E37FE325
:106190000E94463E09F010F40C94DB30ED81FE8144
:1061A0006F817885A981BA818B819C810E94403A58
:1061B0000E94373A0AC0E981FA816B817C81AD8106
:1061C000BE818F8198850E94403AE983FA836B8370
:1061D0007C83003019F00E94EB3C04C0E981FA8115
:1061E0006B817C81088129960895A881B9818A8173
:1061F0009B81E0E0F0E060E87FEB0E94463E58F0D3
:10620000E0E0F0E060E87FE30E94463E19F010F025
:106210000C940B3105C0EFEFFFEF6FE77FE727C06E
:10622000E881F9816A817B810E947B3C0E948630F3
:106230000E94373A1CC0A881B9818A819B810E9443
:10624000823E4CF0E881F9816A817B810E947B3C2F
:106250000E9436300CC0E881F9816A817B810E94FE
:10626000EB3C0E947B3C0E9436300E94EB3C249623
:1062700008952A970E94963EE0E0E887E987EA873A
:10628000EB87A889B989EC914E2F0E94D53919F076
:106290000E94463AF6CFE0E0EF834B3219F40E94B9
:1062A000463A06C04D3221F4E1E0EF830E94463ABF
:1062B000E0E05E2F4E2F08891989A889B989EC91F1
:1062C0000E944C3A49F4A889B989AC91EEE20E9447
:1062D0008E3B4E2FE03021F0542B0E94463AEDCFFA
:1062E00028893989503019F10E94513AA889B98911
:1062F000AC91AE32E1F00E94573AA885B9858A8503
:106300009B85FF27662777270E94473D0E94853D92
:10631000DF01CB01E0E0F0E060E271E40E94053EC5
:10632000E887F9876A877B870E94513ADFCFE0E0F0
:10633000F0E060E87FE3EC87FD876E877F87A889C0
:10634000B9891197A88BB98BA017B107D0F00E941B
:10635000573AAC85BD858E859F85FF2766277727B1
:106360000E94473D0E94D33DA885B9858A859B85BB
:106370000E94853DE887F9876A877B870E945C3A9F
:10638000DECFA22FB32F2F5F3F4F4C91453619F030
:10639000453409F067C0E0E05E2FEE83A22FB32FF3
:1063A000AC91AD3221F4E1E0EE832F5F3F4FA22F9D
:1063B000B32F2F5F3F4FEC914E2F0E944C3A31F09C
:1063C0000E946C39E40FE0535E2FF1CFE6E2E5174F
:1063D00068F4EF81E03029F0EFEFFFEF6FE77FEF38
:1063E0004AC0EFEFFFEF6FE77FE745C040E2E0E034
:1063F000F0E060E87FE3EC87FD876E877F874030C1
:10640000A9F0EC85FD856E857F85AC85BD858E8583
:106410009F850E94D33DEC87FD876E877F87E52FA0
:10642000E42311F00E945C3A4695E9CFEE81E0301A
:1064300059F0EC85FD856E857F85A885B9858A85AF
:106440009B850E94053E0AC0EC85FD856E857F8593
:10645000A885B9858A859B850E94D33DE887F98701
:106460006A877B87EF81E03011F00E947F39E885F1
:10647000F9856A857B850E949D3E62960895E0912C
:10648000A80DF091A90D6091AA0D7091AB0DADE62C
:10649000BEE486EC91E40E94D03BEE59F8486F4F81
:1064A0007F4FE093A80DF093A90D6093AA0D709310
:1064B000AB0DE62FF72FFF770895EA93E5E8FCE0B0
:1064C000FA93EA930895E881F0E0309708950E94E6
:1064D000713CE050F048E093260AF093270A0895B3
:1064E000A6E2BAE00E94623C3296ED93FC930895D6
:1064F000E091260AF091270AE491F0E00895A6E2DF
:10650000BAE00E94623C3496ED93FC930895A6E2B3
:10651000BAE00E94623C3196ED93FC930895E42F1B
:10652000F52F0E94773BEA5FFD4F0895E42FF52F8A
:10653000E770F070EA0FFB1FE4910895A6E0B2E067
:10654000EE0FFF1FAE0FBF1F0895A6E0B2E00E943E
:10655000723BAE0FBF1F0895A02FBB27E3E2F1E00F
:106560000E94C83B0895AE0FBF1FE0E0F0E0ED933E
:10657000FC930895AE0FBF1FE0E0EC93EDCFAE0F9C
:10658000BF1FE0E0EC930895F0E0A2E0B2E0EE0F70
:10659000FF1FAE0FBF1F0E94623C0895E091260AC4
:1065A000F091270A32960E94713C0895A12FBB27D3
:1065B000E3E2F1E00E94C83B0895E491EC93F6CF4A
:1065C000AE0FBF1FEC91F0E00895A02FB12FE3E2D2
:1065D000F1E00E94C83B0895AE0FBF1F0E94623CCD
:1065E000DF01E22FF32F0895EA0FFB1FE491F0E0A3
:1065F0000895AE0FBF1F0E94623CE20FF31FE491AB
:10660000EA930895E0E0EA93E0CFF695E7953196B6
:10661000EE0FFF1FEA0FFB1F0E94713CFA93EA93F3
:106620000895F695E7953296EE0FFF1FEA0FFB1FD0
:106630000E94713CFA93EA93C8CF3696EA0FFB1F8B
:10664000E491EA93C2CFEB57F34FFA93EA930C9499
:106650005C1EEB57F34FFA93EA930C944E20AE0F67
:10666000BF1FE1E0EC930895EB57F34FFA93EA93E1
:106670000C94CC1EEB57F34FFA93EA930C94B6208C
:10668000AE0FBF1FE2E0EC930895AE0FBF1FEC9179
:10669000EF5F0895EB57F34FFA93EA930C9456216A
:1066A000F0E0A3E2B1E00E94C83B08951A930A9378
:1066B00026CF34970E94713C0E2F1F2F0895E02F94
:1066C000F12F0E94773BE050F84FEA5FFD4F0895AD
:1066D000A2E9B0E0E02FF12FE770F070EA0FFB1FA6
:1066E000E4910895E02FF12F0E94773BEA5FFD4F80
:1066F000089534970E94713C3197EA5FFD4FE08125
:106700000895F0E066277727E093490AF0934A0A54
:1067100060934B0A70934C0A089534970E94713C21
:1067200031970CCF0E94623C66277727E093490A95
:10673000F0934A0A60934B0A70934C0A0895349779
:106740000E94713C319701CFAAE9B0E0E02FF12F10
:10675000E770F070EA0FFB1FE491089534970E94F0
:10676000713C3197EA5FFD4FDF01E091490AF091FA
:106770004A0A60914B0A70914C0AEC930895349741
:106780000E94713C3197A6E0B2E0EE0FFF1FAE0F02
:10679000BF1FE091490AF0914A0A60914B0A70913B
:1067A0004C0AED93FC93089534970E94713C319705
:1067B000A6E0B2E00E94723BAE0FBF1FE091490A13
:1067C000F0914A0A60914B0A70914C0A0E946C3C0D
:1067D000089534970E94713C319708953197E49160
:1067E000E1501E2FE091260AF091270A3396E4919A
:1067F000F0E0A3E5BAE0EE0FFF1FAE0FBF1FED9173
:10680000FD910995E091490AF0914A0A60914B0A7D
:1068100070914C0A0E947E3E0895E091260AF09104
:10682000270A3396E491F0E00895A3E5BAE0EE0F6D
:10683000FF1FAE0FBF1FED91FD910995E091490A31
:10684000F0914A0A60914B0A70914C0AAA81BB816F
:106850008C819D810895EA81FB816C817D81E0932B
:10686000490AF0934A0A60934B0A70934C0AD5CFB9
:10687000A7E6BAE0EE0FFF1FAE0FBF1FED91FD912F
:10688000099508950E94623CDF01E12FF0E00E942B
:10689000723BEA0FFB1F0895ED93FC93E091260AEB
:1068A000F091270A0E94713CF0780895A3E5BAE0C0
:1068B000EE0FFF1FAE0FBF1FED91FD910995E09107
:1068C000490AF0914A0A60914B0A70914C0A089566
:1068D000A6E2BAE00E94623C3497ED93FC939DCF10
:1068E000A881B9818A819B810E94983BFF276627F6
:1068F0007727E093490AF0934A0A60934B0A709312
:106900004C0A8BCFA881B9818A819B810E94A03BD0
:10691000FF2766277727E093490AF0934A0A609396
:106920004B0A70934C0A79CF0E94B83BFF27662729
:106930007727E093490AF0934A0A60934B0A7093D1
:106940004C0A6BCF0E94C03BFF2766277727E09356
:10695000490AF0934A0A60934B0A70934C0A5DCF40
:106960000E94A83BFF2766277727E093490AF09308
:106970004A0A60934B0A70934C0A4FCFA881B981A1
:106980008A819B810E94B03BFF2766277727E0938F
:10699000490AF0934A0A60934B0A70934C0A3DCF20
:1069A000A3E5BAE0EE0FFF1FAE0FBF1FED91FD9103
:1069B0000995A091490AB0914A0A80914B0A909199
:1069C0004C0AE0E0F0E060E070E008950E94983B3F
:1069D000FF2766277727E093490AF0934A0A6093D6
:1069E0004B0A70934C0A19CF0E94A03BFF276627E1
:1069F0007727E093490AF0934A0A60934B0A709311
:106A00004C0A0BCFFF2766277727E093490AF093BC
:106A10004A0A60934B0A70934C0AFFCE0E94F80713
:106A2000E0914D0AF0914E0A60914F0A7091500A20
:106A3000E883F9836A837B830E94F807E0914D0A1B
:106A4000F0914E0A60914F0A7091500A08950E9489
:106A5000F807A0914D0AB0914E0A80914F0A90918B
:106A6000500AE0E0F0E060E070E00895A3E5BAE0ED
:106A7000EE0FFF1FAE0FBF1FED91FD910995089519
:106A8000A6E2BAE00E94623C3896ED93FC9308952A
:106A9000E0934D0AF0934E0A60934F0A7093500AA8
:106AA0000E947408E1E0F0E060E070E0E093490AE1
:106AB000F0934A0A60934B0A70934C0A08950E941F
:106AC000623CDF01E12FF0E031960E94723BEA0F59
:106AD000FB1F08950E94F807E0914D0AF0914E0ABD
:106AE00060914F0A7091500AAA81BB818C819D816F
:106AF0000895A6E2BAE00E94623C3C96ED93FC93B6
:106B000008950E94F807E0914D0AF0914E0A6091B5
:106B10004F0A7091500AE883F9836A837B830C944F
:106B2000F807E881F9816A817B810E947B3CE091D2
:106B30004D0AF0914E0A60914F0A7091500A0E94DE
:106B40007B3C08950E94F807E0914D0AF0914E0AAF
:106B500060914F0A7091500A0E947B3C08950E94F8
:106B6000803C0E947E3DDF01CB01E0E0F0E060E090
:106B70007FE308950E94143DE093490AF0934A0A86
:106B800060934B0A70934C0A48CE66277727E093B0
:106B9000490AF0934A0A60934B0A70934C0A3DCE1F
:106BA000A6E2BAE00E94623C38960895A6E2BAE0F6
:106BB0000E94623C34960895E20FF31FDF01E42F38
:106BC000F52F0895A6E2BAE00E94623C7096ED931C
:106BD000FC93089566277727E883F9836A837B838C
:106BE000EA5FFD4FFA93EA930895E091490AF09124
:106BF0004A0A60914B0A70914C0AEA5FFD4FFA9382
:106C0000EA930895E02FF0E0A5E0B0E00E94C83BD1
:106C10000895F0E0EE0FFF1FE85DF54F0895E09155
:106C2000260AF091270A0E94713CE050F048E09358
:106C3000260AF093270A089532970E94713CABE729
:106C4000BAE0EE0FFF1FAE0FBF1FED91FD9109954A
:106C50000895E091490AF0914A0A0E94723BEC8340
:106C6000FD83AC81BD811497E881F9816A817B81C4
:106C70000E94A23C0895E091490AF0914A0A0E94BC
:106C8000723BE883F983A881B98114970E948D3CF7
:106C900008950E94363BA881B9818A819B810E9418
:106CA000363B0895E981FA816B817C81EA5FFD4F73
:106CB000FA93EA930895EA0FFB1FFA93EA93E9E443
:106CC000FAE0662777270E947B3C0895E12FF0E0E9
:106CD000A5E0B0E00E94C83B0895EA0FFB1FFA93BD
:106CE000EA93EE81FF81688579850E947B3C089557
:106CF000A42FBB27E3E2F1E00E94C83B089522974E
:106D00000E94973EFCCBE091490AF0914A0AED833C
:106D1000FE8383CDA22FBB27E3E2F1E00E94C83BB4
:106D200008950A93E0E0EA930895FA93EA931A9398
:106D3000E22FB6CCA6E2BAE00E94623C7496ED93D4
:106D4000FC9308954A933A931A93E22FA9CCEA81CF
:106D5000FB816C817D81EA5FFD4FFA93EA93089590
:106D600066277727EC87FD876E877F87E0E0E883DB
:106D7000E983EA83EB830895EC81FD816E817F8155
:106D8000A881B9818A819B810E94913E0895AC853A
:106D9000BD858E859F850E94363BEA5FFD4F089535
:106DA000E881F9816A817B81EF5FFF4F6F4F7F4FF1
:106DB000E883F9836A837B83089566277727EC83CA
:106DC000FD836E837F839BCBE22FF32FE00FF11FB8
:106DD000EA5FFD4F0895AE0FBF1FEC91E17008957B
:106DE0000A921A92FA926A937A938A939A93AA933E
:106DF000BA93EA93FA93EFB7EA930895E991EFBF54
:106E0000F991E991B991A9919991899179916991B2
:106E1000F990199009900895A881B981A15EBE4F9B
:106E2000AC910895EA81A881B981EC930895A65F99
:106E3000BE4FE1E0F0E0ED93FC930895E091620035
:106E4000E860E0936200A881B9810895A881B981C2
:106E5000A65FBE4F0E94623C0895A881B981A15EE1
:106E6000BE4FE0E00895AB5EBE4FEC91F0E00895B8
:106E7000A881B981A75FBE4FEC91E1700895A88108
:106E8000B981AD5EBE4FEC91F0E00895A881B98163
:106E9000AC5EBE4FEC91F0E00895E0916200E77FB8
:106EA000E09362000895A15EBE4FE4E0EC93089584
:106EB000A05FBE4FE8EEF3E0ED93FC930895AA8146
:106EC000BB81EC9311960895FA93EA93EC81FD81CE
:106ED000FA93EA930E945C240E2F1F2FE12FF0708B
:106EE00008950C93AA81BB81A45FBE4F0895ED93D2
:106EF000FC93AA81BB81D7CFAA81BB81A75FBE4F7C
:106F0000EC91E1700895AA81BB81AD5EBE4FEC911A
:106F1000F0E00895AA81BB81AC5EBE4FEC91F0E039
:106F20000895E0916200E860E09362000895E02F28
:106F3000F0E03796AD81BE81EA0FFB1F0895AB816B
:106F4000BC81ED91AB83BC830895E02FF0E03796D0
:106F50000895EF81F0E037960895EC93EF81F0E02B
:106F60000895A75FBE4FEC91E1700895AD5EBE4FEE
:106F7000EC91F0E00895AC5EBE4FEC91F0E0089526
:106F8000E981FA813196E983FA8331970895AB81DB
:106F9000BC81AE0FBF1FEC910895E12FF0E0AF81EF
:106FA000B885EA0FFB1F08953196EA5FFD4FE08137
:106FB0000895EE81F0E0EE0FFF1F34960895EE8104
:106FC000F0E0EE0FFF1F0895EC91F0E03097089588
:106FD000AE85BF85A05EBE4FF7CFAE85BF85A65FED
:106FE000BE4F0E94623CFA93EA93E889F989FA93CA
:106FF000EA930E945C2430970895AE85BF8515966C
:10700000EC91FE2FE0E00895AE85BF851496EC91DB
:10701000F0E00895EE85FF85A181AA93EF85F889B8
:107020000895A381AA931A930A930895E989FA8986
:10703000A681AA93EA89FB89FA93EA930C94CE1F5E
:10704000AE85BF85A15EBE4FE6E0EC930895AE85A8
:10705000BF85A05EBE4FE0E0EC930895AE85BF858E
:107060001196AC910895AE85BF851296EC91089566
:10707000AE85BF851496EC91FE2FE0E00895AE85B5
:10708000BF851596EC91F0E00895EA0FFB1FEC87A1
:10709000FD87EE0FFF1F0895EC85FD85AA85BB8552
:1070A000AE17BF070895EA85FB85EE0FFF1FE8873F
:1070B000F9870895E885F9853396AE85BF85EA0F8F
:1070C000FB1F0895EF81F0E0A885B985EA0FFB1F4B
:1070D0000895EC93E885F9853496AE85BF85EA0F6F
:1070E000FB1F0895EA85FB853196EA87FB870895A3
:1070F000EC85FD85EE0FFF1F33960895FA93EA9312
:10710000E889F989FA93EA930E945C244E2F5F2F55
:10711000EFCFAE85BF85AE0FBF1FE52FF070EC93AC
:10712000EC85FD85EE0FFF1F3496AE85BF85AE0F53
:10713000BF1F4C93EC85FD85EE0FFF1F359608951C
:10714000F695E795AA85BB85AE17BF070895EA8532
:10715000FB850E94723BE887F9870895AE85BF855D
:10716000A45FBE4FE8E0F0E0ED93FC93E1E0EE8336
:107170000895AE85BF85AE0FBF1FEC910895A88519
:10718000B985EA0FFB1F3196EA5FFD4F0895AE8582
:10719000BF85A55EBE4FEC910895AE85BF85A45E08
:1071A000BE4F0E94623C0895AE85BF85A05EBE4F73
:1071B000E0E00895AE85BF85A15EBE4FE6E008958C
:1071C000A881B981A15FBE4FE2E0EC930895EE0F74
:1071D000FF1FEA0FFB1F0E94713C08950E94623C52
:1071E0003196ED93FC93089524971A930A9308958A
:1071F000AE81BF811196AE83BF8311970895E0E001
:10720000F0E060E271E40E94053EA0E0B0E080E0C2
:107210009FE30E94853D0E947B3C0C94233B0E948F
:10722000053E0E94143D1E2F0895E12FE05DEC9372
:10723000E12F08950E94803C0E947E3DE987FA87F5
:107240006B877C870895AE81BF81E0E0EC93089561
:10725000AB81BC818D819E81E0E0F0E060E271E471
:107260000E94D33DEB83FC836D837E830895EB8185
:10727000FC816D817E81AB85BC858D859E850E945C
:10728000463E0895AB85BC858D859E85E0E0F0E0A7
:1072900060E271E40E94053EEB87FC876D877E8784
:1072A0000895AF81B8851196AF83B8871197089577
:1072B000EF81F8853196EF83F887319708953A93F7
:1072C000EBA1FCA1FA93EA930C940A28A42FEAE01C
:1072D000EA9FE02D4E2F0895A52FEAE0EA9FE02DCA
:1072E0000895ACA1BDA11497ACA3BDA314960895B5
:1072F000EA93EBA1FCA1FA93EA930C940A28E8859F
:10730000F9856A857B850E94EB3CE887F9876A8767
:107310007B870895EE81FF813196EE83FF8331975D
:107320000895E885F9856A857B850E947B3C5A93A0
:107330000895EE83FF83FA93EA930E94A93A0E2FF1
:10734000089522971A930A93DE010E94323B0A2F76
:107350001B2FDE0116960E94323B0E94623CEA839C
:10736000FB83DE0114960E94323B0E94623CFA933A
:10737000EA931A930A93FE013696FA93EA930895D4
:107380002A930E94733AE0300895FE013C96FA93E6
:10739000EA93EF85F889FA93EA930C94CB2BE98969
:1073A000FA892591E98BFA8B0895EA930E94733A42
:1073B000E0300895AF85B8891497AF87B88B1496DD
:1073C0000D911C910895E0E0F0E060E87FE30E94F9
:1073D000803C0E947E3D0895EE83FF836887798715
:1073E000AE81BF81888599850E94D33DEA83FB8366
:1073F0006C837D8308950E947B3C0E94852DAC8127
:10740000BD818E819F810E94D33D0E947B3C0C9464
:10741000212E0E94803C0E947E3DED83FE836F837F
:1074200078870895ED81FE816F8178850E94EB3C1D
:10743000ED83FE836F8378870895ED81FE816F81F0
:107440007885AD81BE818F8198850E94D33D089556
:107450000E94D33DAEE4BFE88AE491E40E94853DFA
:1074600008950E94053E0E947B3C0C94FF2FABEDDB
:10747000BFE089EC9FE30E94803C0E947E3D08951E
:107480000E94053E0E947B3C0C943630E889F989C5
:107490003196E88BF98B0895EA930E946B3AE030BD
:1074A0000895E889F9893197E88BF98B0895A889BF
:1074B000B989EC91E0530895AC85BD858E859F8593
:1074C000E0E0F0E060E271E40E94D33DEC87FD87EC
:1074D0006E877F870895E1E0F991F03310F0FA3379
:1074E00008F0EE270895E1E0F991F03229F0F93043
:1074F00010F0FE3008F0EE270895E991F991A99176
:10750000B991CD016D916623E9F7119761916D9362
:107510006623E1F7FC010895E991F991A991B991E8
:107520006D917191671721F46623D1F7EE270895C5
:10753000671BE1F3E1E008F4E2500895E991F99165
:10754000A991B991CD0161916D936623E1F7FC0199
:107550000895A991B991EE27FF276D91662311F047
:107560003196FBCF0895AA27BB27E991F9910590A1
:10757000002011F01196FBCFFD01089524975F9331
:107580009F81992311F4289602C312F4289605C30B
:107590004F9342E48E81BD81AC8188839983AA8315
:1075A000BB83FD01BC01AC81BD818E819F812DD348
:1075B00088819981AA81BB81A8D22DD27A9511D2D6
:1075C00088819981AA81BB81AE27A87F21F4BF174A
:1075D0008607970729F04A9519F0DF01CB01DDCF27
:1075E0004F915F91289608957B816A81F981E881A6
:1075F00077FB770F67FD7160972F9E5781F078F0CA
:10760000983190F4AA27BB27882708948795B795C7
:10761000A7959A95D1F7EA23FB23682305C0E89440
:107620007727EE27FF2766276F77769508F460683F
:1076300077F9A991B99189919991EA17FB076807A0
:10764000790797FB0895D0DF09F40895F6F79FEBCB
:1076500005C0CADF09F40895F6F39FE3AA27BB2704
:1076600080E853C20024AF0DB01D0895EA0FFB1F40
:10767000681F791F0895EA1BFB0B680B790B0895AF
:10768000EA23FB23682379230895EA2BFB2B682B3D
:10769000792B0895EA27FB27682779270895E09535
:1076A000F09560957095EF5FFF4F6F4F7F4F089596
:1076B000EE230E2EFD01BC0131F0EE0FFF1F661F01
:1076C000771F0A94D1F70895EE230E2EFD01BC0119
:1076D00031F075956795F795E7950A94D1F7089578
:1076E000EE0FFF1FEE0FFF1FEE0FFF1F0895F69521
:1076F000E795F695E795F695E7950895FE2FFF0F28
:10770000FF0B6F2F7F2F08956F2F660F660B762F5D
:107710000895E095F095609570950895EA17E1E079
:1077200009F0EE270895EA17E1E009F4EE2708953D
:10773000EA17FB0768077907E1E009F0EE270895EB
:10774000EA17FB0768077907E1E009F4EE270895D7
:10775000EA17FB0768077907E1E00CF4EE270895C4
:10776000AE17BF0786079707E1E00CF4EE270895F0
:10777000AE17BF0786079707E1E00CF0EE270895E4
:10778000EA17FB0768077907E1E00CF0EE27089598
:10779000FA9FF02DEB9FF00DEA9FE02DF10D08957B
:1077A0007A9F702D6B9F700DF89F700DE99F700D83
:1077B0006A9F602D710DFB9F600D711DE89F600D2C
:1077C000711D8827FA9FF02D610D781FEB9FF00D3A
:1077D000611D781FEA9FE02DF10D681F781F089545
:1077E0005ED0DEDF0EF45BDF0895002498E0AA0F80
:1077F000001C0E1A10F40E0E01C0A1609A95B9F784
:10780000EA2FA02D08953FD0F0DF0EF4E195089502
:107810003F934F935F93002411243327442750E272
:10782000AA0FBB1F881F991F001C111C331F441F68
:107830000E1A1F0A360B470B28F40E0E1F1E361F9A
:10784000471F01C0A1605A9559F7FD01BC01D00145
:10785000832F942F5F914F913F91089520D0D8DFCF
:107860000EF41DDF0895E894A7FF02C0A195689467
:10787000E7FDE195BADFEA2F0EF4E1950895C8DF40
:10788000FD01BC010895E894E7FF02C0E19568940A
:10789000A7FF04C0A19500F8039400FA0895E894A6
:1078A00077FF02C0FCDE689497FF0BC00024A09510
:1078B000B095809590951196801D901D00F80394C9
:1078C00000FA0895ED91FC9111970895ED91FD91C5
:1078D0006D917C9113970895ED93FD936D937C9337
:1078E00008950590F491E02D089505901590659107
:1078F0007491F00108957A936A93FA93EA93089544
:10790000182E862F612D192E972F712D1B2EBF2F0C
:10791000F12D1A2EAE2FE12D0895129603D07F2F50
:107920006E2F1297119602D0FE2F1197E199FECF7C
:10793000FF93FFB7F894AEBBBFBBE09AEDB3FFBFB8
:10794000FF9108950AD012960E2E1F2EE62FF72FC4
:1079500004D0E02DF12D1297089507D01196EF93E2
:10796000EF2F03D0EF9111970895E199FECF9FB7C4
:10797000F894AEBBBFBBE09A8DB3E81719F0EDBB2E
:10798000E29AE19A9FBF0895992761916D930197BB
:10799000E1F70895A991B991E991F99169917991E6
:1079A00077FB660F771F88277E57880B7D938C9314
:1079B0007EE7769567957EF00895A991B991E99152
:1079C000F9916991799177FB660F771F7A0F769518
:1079D00067950EF0089530976040704009F0705838
:1079E000089550E8572711F45F93D1C05F3F31F0FD
:1079F000660F000C57956795752F08955F930020CB
:107A00000AF0CBC0BEC050E8192E1522880F991F6E
:107A10009527550F879550E8072E0522660F771F8B
:107A20007527550F679508955F93F5DF703818F047
:107A30007F3F08F4ACC056E1571B92F45195583083
:107A400028F0EFEFFFEF6FEF7FE71AC0772755239E
:107A5000B9F0EE0FFF1F661F771F5A95D1F710C0C0
:107A60007727583028F0EF2FF62F672F5850F9CF8F
:107A7000552331F076956795F795E7955A95D1F7A7
:107A800000200AF40CDE5F910895689401C0E89428
:107A9000309760407040B1F0002426F0772312F454
:107AA0000094FDDD172E7EE1112032F07A95EE0F65
:107AB000FF1F661F111CF9CFEF2FF62F612D5F936B
:107AC00090DF5F9108955E2FEA2FA52F5F2FFB2F88
:107AD000B52F562F682F852F572F792F952F502D83
:107AE000012C152E0895EA0FFB1F681F0895E095DD
:107AF000F0956095EF5FFF4F6F4F08955F9383DFC1
:107B0000903871F150E8152604C05F937CDF9038FF
:107B100039F1703821F1572F591B13F112F4D3DFCB
:107B2000FACF583118F0AA27BB278827583028F0F9
:107B3000AB2FB82F88275850F9CF552329F08695B9
:107B4000B795A7955A95D9F7502D512562F0CBDFFF
:107B500038F46795F795E795739513F41EC0B3DF76
:107B600040DF5F910895EA1BFB0B680B81F010F476
:107B70000094BDDF6623A2F3EE0FFF1F661F7A9508
:107B8000CBF7EFEFFFEF6FE77FEF5F910895EE2701
:107B9000FF27662777275F910895EFEFFFEF6FE7E5
:107BA0007FE75F9108955F932EDF703881F39038FF
:107BB00071F301240894791F23F44CF300200AF395
:107BC000ECCF3F934F93112433274427552798E157
:107BD000330F441F551FEE1FFF1F661F30F43A0F6F
:107BE0004B1F581FE11DF11D611D9A9589F74F919B
:107BF0003F9166232AF0550FEE1FFF1F661F02C03C
:107C00007395E3F2EEDE5F9108955F93FCDE7038CA
:107C100019F4112012F6B5CF903809F4B8CF012429
:107C20000894970B1BF4D4F30020F4CF792F6695BA
:107C3000F795E7958695B795A7954F931124442717
:107C4000552798E1AE17BF07860728F0AE1BBF0B7C
:107C5000860B089401C08894111C441F551FAA1F4D
:107C6000BB1F881F9A9571F7E12DF42F652FA695FC
:107C7000E91FF91F691F4F9166232AF0EE0FFF1FBE
:107C8000661F7A955BF2ADDE5F91089599239AF0B5
:107C9000772342F0971748F029F4AE17BF078607FD
:107CA00020F031F098948894089598940894089559
:107CB0001894889408957723C2F7971798F3A9F733
:107CC000EA17FB07680788F399F3ECCFDFDFE1E001
:107CD00011F008F0EE270895D9DFE1E011F008F483
:107CE000EE270895D3DFE1E009F008F0EE270895CC
:107CF000CDDFE1E009F008F4EE2708953097604009
:107D000070400895109780409040089500240A160E
:107D10000B06080609060895EA17FB0768077907A6
:107D20000895AE17BF078607970708955A934A9399
:107D30003A932A931A930A9308955D814C813B816B
:107D40002A81198108810895AC0FBD1F05900D92FD
:107D50008A95E1F70895FFFFFFFFFFFFFFFFFFFF99
:107D6000FFFFFFFFFFFFFFFFFFFFFFFFFFFFFFFF23
:107D7000FFFFFFFFFFFFFFFFFFFFFFFFFFFFFFFF13
:107D8000FFFFFFFFFFFFFFFFFFFFFFFFFFFFFFFF03
:107D9000FFFFFFFFFFFFFFFFFFFFFFFFFFFFFFFFF3
:108000002F164A0129002C002D0042012A004901A7
:108010000000000000000000504143353133305F64
:1080200030000000000000000000590000130003B1
:1080300044493101000000020000000000034449EF
:108040003202000000020000000000034449330334
:108050000000000200000000000344493404000056
:108060000002000000000003444935050000000242
:108070000000000000034449360600000002000032
:108080000000000344493707000000020000000020
:10809000000344493808000000020000000000030B
:1080A000444F310900000002000000000003444F6B
:1080B000320A00000002000000000003444F330BAE
:1080C00000000002000000000003444F340C0000D8
:1080D0000002000000000003444F350D00000002C4
:1080E000000000000003444F360E000000020000B4
:1080F00000000003444F370F0000000200000000A2
:108100000003444F3810000000020000000000038C
:108110004449730100000004000000000003444FC4
:1081200073020000000400000000000C506F77652F
:10813000724D6F6E69746F721100000002000000D2
:1081400000000100002C010400000000FC5BD700CF
:10815000FC5BD70028000000AC8E4200D8DCD600C3
:108160001817C90010DDD600110000FF60000000E4
:10817000280000001700000094844100505CD700E4
:10818000010000000400000016000000B0BBD60093
:1081900014000000000000001400000016000000A1
:1081A000F0C9D600140000000853C90014000000F4
:1081B0007A0000000C67420001000000EC17050B7C
:1081C0000000000000000000EC17050B000000009C
:1081D0004000000040000000C00000000100180046
:1081E0000000AC012800000040000000400000003A
:1081F0000100180000000000003000000000000036
:10820000FFFFFFFFFFFFFFFFFFFFFFFFFFFFFFFF7E
:10821000FFFFFFFFFFFFFFFFFFFFFFFFFFFFFFFF6E
:10822000FFFFFFFFFFFFFFFFFFFFFFFFFFFFFFFF5E
:10823000FFFFFFFFFFFFFFFFFFFFFFFFFFFFFFFF4E
:10F000000C944F790C9400780C9400780C94007850
:10F010000C9400780C9400780C9400780C94007890
:10F020000C9400780C9400780C9400780C94007880
:10F030000C9400780C9400780C9400780C94007870
:10F040000C94F9790C9400780C9400780C94007866
:10F050000C9400780C9400780C9400780C94007850
:10F060000C9400780C9400780C9400780C94007840
:10F070000C9400780C9400780C94567A0C940078D8
:10F080000C949A7A0C9400780C940078010204088D
:10F0900010204080FEFDFBF7EFDFBF7F0000C0C106
:10F0A000C1810140C30103C00280C241C60106C044
:10F0B0000780C7410500C5C1C4810440CC010CC014
:10F0C0000D80CD410F00CFC1CE810E400A00CAC1D4
:10F0D000CB810B40C90109C00880C841D80118C0C4
:10F0E0001980D9411B00DBC1DA811A401E00DEC144
:10F0F000DF811F40DD011DC01C80DC411400D4C134
:10F10000D5811540D70117C01680D641D20112C053
:10F110001380D3411100D1C1D0811040F00130C023
:10F120003180F1413300F3C1F28132403600F6C143
:10F13000F7813740F50135C03480F4413C00FCC113
:10F14000FD813D40FF013FC03E80FE41FA013AC0D3
:10F150003B80FB413900F9C1F88138402800E8C103
:10F16000E9812940EB012BC02A80EA41EE012EC043
:10F170002F80EF412D00EDC1EC812C40E40124C033
:10F180002580E5412700E7C1E68126402200E2C153
:10F19000E3812340E10121C02080E041A00160C063
:10F1A0006180A1416300A3C1A28162406600A6C143
:10F1B000A7816740A50165C06480A4416C00ACC113
:10F1C000AD816D40AF016FC06E80AE41AA016AC0D3
:10F1D0006B80AB416900A9C1A88168407800B8C1C3
:10F1E000B9817940BB017BC07A80BA41BE017EC043
:10F1F0007F80BF417D00BDC1BC817C40B40174C033
:10F200007580B5417700B7C1B68176407200B2C152
:10F21000B3817340B10171C07080B041500090C1A2
:10F2200091815140930153C052809241960156C042
:10F2300057809741550095C1948154409C015CC012
:10F240005D809D415F009FC19E815E405A009AC1D2
:10F250009B815B40990159C058809841880148C002
:10F26000498089414B008BC18A814A404E008EC142
:10F270008F814F408D014DC04C808C41440084C132
:10F2800085814540870147C046808641820142C052
:10F2900043808341410081C1808140400000F89457
:10F2A000EE27ECBBF1E0F5BFF2E0F5BFE0936C00B8
:10F2B000F8E1F1BDE1BD8DE0A2E0BB27ED938A95B9
:10F2C000E9F780E090E1A0E0B1E0ED930197E9F784
:10F2D000ECE9F2EF85919591009761F0A591B591D8
:10F2E00005901590BF01F00105900D920197E1F78F
:10F2F000FB01F0CFEFEFEDBFE0E1EEBFC0E0D2E009
:10F300000C94BF7B09801A80EB81FC81B881B0939B
:10F310006800E895E0916800E170E1F725960895AE
:10F320001A930A93F8940E944D7CE3E00E94587C63
:10F3300000E010E00038E0E01E07A8F4E02FF12F15
:10F34000EE0FFF1FFA93EA93AC81BD81ED91FD9121
:10F35000AC83BD83FA93EA93E1E0EA930E94827959
:10F360000F5F1F4FE7CF0E944D7CE5E00E94587C65
:10F37000789419810881269608950E94B27C0FEF37
:10F380001FEF20E030E0EE81FF812E173F0758F598
:10F39000E02FF12FFE2FE0E0FF93EF93ECE9F0EF89
:10F3A000FF93EF93E12FF070FF93EF93E22FF32F92
:10F3B000AC81BD81AE0FBF1FEC91F0E0AF91BF916A
:10F3C000EA27FB27AF91BF91EE0FFF1FEA0FFB1F4C
:10F3D0000E94A97CAF91BF91EA27FB270E2F1F2F18
:10F3E0002F5F3F4FD0CFE02FF12F0E94B77C2896A0
:10F3F00008956A937A93AA93BA93EA93FA93EFB72C
:10F40000EA93E6E0E2BFE0911703F0911803609100
:10F41000190370911A03EF5FFF4F6F4F7F4FE09317
:10F420001703F09318036093190370931A03A895B8
:10F43000E0910E03F0910F03309779F1AEE0B3E065
:10F440000E94A57C3197ED93FC93309731F5E091C4
:10F450001303F0E0E230A0E0FA0721F4E5E0E093E6
:10F4600013031BC0E330A0E0FA0721F4E0E0E093CF
:10F47000130313C0E130A0E0FA0721F4E6E0E093C3
:10F4800013030BC0E430A0E0FA0739F4E0E0E093A6
:10F490001303E09314030E94657CE991EFBFF99197
:10F4A000E991B991A9917991699118950E946B7C24
:10F4B0000A9300919C00A0911303E2E0EA1778F10F
:10F4C000A0911303A230A1F0031571F40093000280
:10F4D000E1E0F0E0E0930903F0930A030E94727CFC
:10F4E000E2E0E093130303C0E3E0E093130317C0EB
:10F4F000E0910903F0910A03E930A1E0FA0760F412
:10F50000E0910903F0910A03E050FE4F0083A9E067
:10F51000B3E00E94787C03C0E0E0E0931303E09145
:10F520000D03F0E0E0930E03F0930F0309910E94A6
:10F530007E7C18950E946B7CA0911303A43069F522
:10F54000A9E0B3E00E94A57CFF93EF93ABE0B3E0AA
:10F550000E94A57CAF91BF91AE17BF0770F4E091F8
:10F560000903F0910A03E050FE4FE081E0939C0014
:10F57000A9E0B3E00E94787C10C00E94657CE0E0C6
:10F58000E0931303E0E0F0E0E0930903F0930A0353
:10F59000E0916200E77FE09362000E947E7C189514
:10F5A000E881E0930002E2E0E0930102E2E0F0E0B3
:10F5B000E0930B03F0930C03E4E0E0931303E8EE15
:10F5C000F3E0E0930E03F0930F03E1E0F0E0E0934B
:10F5D0000903F0930A030E94857CE881E0939C0074
:10F5E0002196089522970E94B37CEC85E093000257
:10F5F00030920102E1E0E0930202EB85E093030226
:10F60000E985E0930402EA85E0930502ED81E09349
:10F610000602E885F0E0E230A0E0FA07A9F4EE8106
:10F62000FF81EB83FC8300E0ED810E1768F4E02F8F
:10F630000E948B7CEB81FC813196EB83FC833197BC
:10F64000E491EC930F5FF0CFED81F0E037960E94EC
:10F65000917C1E2F2F2FED810E948B7CE22FF0706A
:10F66000EC93ED81F0E03896E050FE4F1083ED8191
:10F67000F0E03996E0930B03F0930C03E4E0E093A1
:10F680001303E8EEF3E0E0930E03F0930F03E1E0E1
:10F69000F0E0E0930903F0930A030E94857CEC8577
:10F6A000E0939C000E94B87C2D960895AA81A23018
:10F6B00079F4E981F070FA93EA93E7E0F2E0FA93E3
:10F6C000EA930E949079E981F070EBBBE0E0E5BB42
:10F6D000239608950E94B27CE0E0E0931303E0914A
:10F6E0001403F0E0309711F00C94BB7BE091090318
:10F6F000F0910A030E94917C309711F00C94BB7B2F
:10F70000B0910502A0E0E0910402F0E0EA0FFB1FD7
:10F710000E2F1F2FE0910202F0E03097E1F4B0913C
:10F720000802E0910702F0E0EA0FFB1F2E2F3F2FA7
:10F73000E0910102EA93E0910602EA933A932A9358
:10F74000E0910302EA931A930A93E0910902EA9383
:10F750000E94F27A10C0E130A0E0FA0761F4E09173
:10F760000302EA931A930A930E94567BE0910102E6
:10F77000EA930E94D07A0E94B77C24960895249739
:10F78000E0E0EBBBEFEFEABBE0E0E5BBEFEFE4BBB3
:10F79000E0EFE2BBE3E0E1BBE0B3E095AE2FEA2FA0
:10F7A000E295EF703E2E332011F40C94D97B0C942B
:10F7B0000000E0E0E8BBE7BBE3B9E2B9BAD0B9D0FA
:10F7C000E1E0E0936500E0E1E0936400E4E0E3BFA2
:10F7D000E6E0E2BFE0E0E1BFE1E0E7BFE0E0E093C8
:10F7E0007D00E0E8E8B9E0E0E0BDE2E0E0939B0006
:10F7F000E8EDE0939A00E6E0E0939D00E0E0E0931E
:10F800009800EFE0E0939900929AE2E0E0930D0314
:10F810007894EFEFEBBBE5BBE0911703F091180391
:10F820006091190370911A03E883F9836A837B83DB
:10F83000E881F9816A817B81A0911703B091180357
:10F840008091190390911A030E94A07CEAEFF0E0E6
:10F8500060E070E00E94AD7C94F4E894919B689421
:10F86000A2B3A1F9A2BBE0911703F0911803609134
:10F87000190370911A03E883F9836A837B83E0910B
:10F880001303F0E0309731F0E530A0E0FA0711F40F
:10F890000E946A7BCDCF2496FFCFEC81FD81FE2FA5
:10F8A000E0E0FA93EA93E0E0F0E0FA93EA93089557
:10F8B000EA930E948279E0E0F0E0FA93EA93FA9307
:10F8C000EA93E1E1EA930C948279E0916500EF70AC
:10F8D000E09365000895AA93BA93EA93FA93EFB779
:10F8E000EA930895E0916200E860E0936200089571
:10F8F0000E94A57C3196ED93FC930895E991EFBFAA
:10F90000F991E991B991A9910895E0916500E061BB
:10F91000E0936500E7CFF0E03796E050FE4FDF015F
:10F920000895FA93EA93E0E0F2E0FA93EA930C94F4
:10F93000BD79EFE0E0936200E8E0E09361000895B4
:10F94000AE1BBF0B860B970B0895ED91FC911197A1
:10F9500008950590F491E02D0895EA17FB076807D4
:10F96000790708953A932A931A930A9308953B814D
:10F970002A81198108810895FFFFFFFFFFFFFFFF24
:10F98000FFFFFFFFFFFFFFFFFFFFFFFFFFFFFFFF87
:10F99000FFFFFFFFFFFFFFFFFFFFFFFFFFFFFFFF77
:10F9A000FFFFFFFFFFFFFFFFFFFFFFFFFFFFFFFF67
:10F9B000FFFFFFFFFFFFFFFFFFFFFFFFFFFFFFFF57
:10FC00000C94000009801A80EB81FC81B881B093CC
:10FC10006800E895E0916800E170E1F725960895A5
:10FC20001A930A93F894EC81FD81FE2FE0E0FA9399
:10FC3000EA93E0E0F0E0FA93EA93E3E0EA930E94CB
:10FC4000027EE0E0F0E0FA93EA93FA93EA93E1E1CE
:10FC5000EA930E94027E00E010E00038E0E01E0718
:10FC6000A8F4E02FF12FEE0FFF1FFA93EA93AC8177
:10FC7000BD81ED91FD91AC83BD83FA93EA93E1E000
:10FC8000EA930E94027E0F5F1F4FE7CFEC81FD8158
:10FC9000FE2FE0E0FA93EA93E0E0F0E0FA93EA93D3
:10FCA000E5E0EA930E94027EE0E0F0E0FA93EA9356
:10FCB000FA93EA93E1E1EA930E94027E7894198133
:10FCC000088126960895FFFFFFFFFFFFFFFFFFFF5C
:10FCD000FFFFFFFFFFFFFFFFFFFFFFFFFFFFFFFF34
:10FCE000FFFFFFFFFFFFFFFFFFFFFFFFFFFFFFFF24
:10FCF000FFFFFFFFFFFFFFFFFFFFFFFFFFFFFFFF14
:10FD0000FFFFFFFFFFFFFFFFFFFFFFFFFFFFFFFF03
:00000001FF
